Archive member included because of file (symbol)

/opt/altera/altera12.1/nios2eds/bin/gnu/H-i686-pc-linux-gnu/bin/../lib/gcc/nios2-elf/4.1.2/mno-hw-mul/libgcc.a(lib2-divmod.o)
                              obj/default/main.o (__umodsi3)
/opt/altera/altera12.1/nios2eds/bin/gnu/H-i686-pc-linux-gnu/bin/../lib/gcc/nios2-elf/4.1.2/mno-hw-mul/libgcc.a(lib2-mul.o)
                              obj/default/main.o (__mulsi3)
../snake_software_bsp//libhal_bsp.a(alt_load.o)
                              ../snake_software_bsp//obj/HAL/src/crt0.o (alt_load)
../snake_software_bsp//libhal_bsp.a(alt_main.o)
                              ../snake_software_bsp//obj/HAL/src/crt0.o (alt_main)
../snake_software_bsp//libhal_bsp.a(alt_usleep.o)
                              obj/default/main.o (usleep)
../snake_software_bsp//libhal_bsp.a(alt_sys_init.o)
                              ../snake_software_bsp//libhal_bsp.a(alt_main.o) (alt_irq_init)
../snake_software_bsp//libhal_bsp.a(altera_avalon_jtag_uart_fd.o)
                              ../snake_software_bsp//libhal_bsp.a(alt_sys_init.o) (altera_avalon_jtag_uart_read_fd)
../snake_software_bsp//libhal_bsp.a(altera_avalon_jtag_uart_init.o)
                              ../snake_software_bsp//libhal_bsp.a(alt_sys_init.o) (altera_avalon_jtag_uart_init)
../snake_software_bsp//libhal_bsp.a(altera_avalon_jtag_uart_ioctl.o)
                              ../snake_software_bsp//libhal_bsp.a(altera_avalon_jtag_uart_fd.o) (altera_avalon_jtag_uart_ioctl)
../snake_software_bsp//libhal_bsp.a(altera_avalon_jtag_uart_read.o)
                              ../snake_software_bsp//libhal_bsp.a(altera_avalon_jtag_uart_fd.o) (altera_avalon_jtag_uart_read)
../snake_software_bsp//libhal_bsp.a(altera_avalon_jtag_uart_write.o)
                              ../snake_software_bsp//libhal_bsp.a(altera_avalon_jtag_uart_fd.o) (altera_avalon_jtag_uart_write)
../snake_software_bsp//libhal_bsp.a(alt_alarm_start.o)
                              ../snake_software_bsp//libhal_bsp.a(altera_avalon_jtag_uart_init.o) (alt_alarm_start)
../snake_software_bsp//libhal_bsp.a(alt_busy_sleep.o)
                              ../snake_software_bsp//libhal_bsp.a(alt_usleep.o) (alt_busy_sleep)
../snake_software_bsp//libhal_bsp.a(alt_close.o)
                              ../snake_software_bsp//libhal_bsp.a(alt_main.o) (close)
../snake_software_bsp//libhal_bsp.a(alt_dcache_flush_all.o)
                              ../snake_software_bsp//libhal_bsp.a(alt_load.o) (alt_dcache_flush_all)
../snake_software_bsp//libhal_bsp.a(alt_dev.o)
                              ../snake_software_bsp//libhal_bsp.a(alt_sys_init.o) (alt_dev_list)
../snake_software_bsp//libhal_bsp.a(alt_dev_llist_insert.o)
                              ../snake_software_bsp//libhal_bsp.a(alt_sys_init.o) (alt_dev_llist_insert)
../snake_software_bsp//libhal_bsp.a(alt_do_ctors.o)
                              ../snake_software_bsp//libhal_bsp.a(alt_main.o) (_do_ctors)
../snake_software_bsp//libhal_bsp.a(alt_do_dtors.o)
                              ../snake_software_bsp//libhal_bsp.a(alt_main.o) (_do_dtors)
../snake_software_bsp//libhal_bsp.a(alt_errno.o)
                              ../snake_software_bsp//libhal_bsp.a(alt_close.o) (alt_errno)
../snake_software_bsp//libhal_bsp.a(alt_icache_flush_all.o)
                              ../snake_software_bsp//libhal_bsp.a(alt_load.o) (alt_icache_flush_all)
../snake_software_bsp//libhal_bsp.a(alt_iic.o)
                              ../snake_software_bsp//libhal_bsp.a(altera_avalon_jtag_uart_init.o) (alt_ic_isr_register)
../snake_software_bsp//libhal_bsp.a(alt_iic_isr_register.o)
                              ../snake_software_bsp//libhal_bsp.a(alt_iic.o) (alt_iic_isr_register)
../snake_software_bsp//libhal_bsp.a(alt_io_redirect.o)
                              ../snake_software_bsp//libhal_bsp.a(alt_main.o) (alt_io_redirect)
../snake_software_bsp//libhal_bsp.a(alt_irq_entry.o)
                              ../snake_software_bsp//libhal_bsp.a(alt_iic_isr_register.o) (alt_irq_entry)
../snake_software_bsp//libhal_bsp.a(alt_irq_handler.o)
                              ../snake_software_bsp//libhal_bsp.a(alt_iic_isr_register.o) (alt_irq_handler)
../snake_software_bsp//libhal_bsp.a(alt_irq_vars.o)
                              ../snake_software_bsp//libhal_bsp.a(alt_iic.o) (alt_irq_active)
../snake_software_bsp//libhal_bsp.a(alt_open.o)
                              ../snake_software_bsp//libhal_bsp.a(alt_io_redirect.o) (open)
../snake_software_bsp//libhal_bsp.a(alt_release_fd.o)
                              ../snake_software_bsp//libhal_bsp.a(alt_close.o) (alt_release_fd)
../snake_software_bsp//libhal_bsp.a(alt_tick.o)
                              ../snake_software_bsp//libhal_bsp.a(altera_avalon_jtag_uart_init.o) (_alt_tick_rate)
../snake_software_bsp//libhal_bsp.a(altera_nios2_irq.o)
                              ../snake_software_bsp//libhal_bsp.a(alt_sys_init.o) (altera_nios2_irq_init)
../snake_software_bsp//libhal_bsp.a(alt_exception_entry.o)
                              ../snake_software_bsp//libhal_bsp.a(alt_irq_entry.o) (alt_exception)
../snake_software_bsp//libhal_bsp.a(alt_find_dev.o)
                              ../snake_software_bsp//libhal_bsp.a(alt_open.o) (alt_find_dev)
../snake_software_bsp//libhal_bsp.a(alt_find_file.o)
                              ../snake_software_bsp//libhal_bsp.a(alt_open.o) (alt_find_file)
../snake_software_bsp//libhal_bsp.a(alt_get_fd.o)
                              ../snake_software_bsp//libhal_bsp.a(alt_open.o) (alt_get_fd)
/opt/altera/altera12.1/nios2eds/bin/gnu/H-i686-pc-linux-gnu/bin/../lib/gcc/nios2-elf/4.1.2/../../../../nios2-elf/lib/mno-hw-mul/libc.a(lib_a-atexit.o)
                              ../snake_software_bsp//libhal_bsp.a(alt_main.o) (atexit)
/opt/altera/altera12.1/nios2eds/bin/gnu/H-i686-pc-linux-gnu/bin/../lib/gcc/nios2-elf/4.1.2/../../../../nios2-elf/lib/mno-hw-mul/libc.a(lib_a-exit.o)
                              ../snake_software_bsp//libhal_bsp.a(alt_main.o) (exit)
/opt/altera/altera12.1/nios2eds/bin/gnu/H-i686-pc-linux-gnu/bin/../lib/gcc/nios2-elf/4.1.2/../../../../nios2-elf/lib/mno-hw-mul/libc.a(lib_a-impure.o)
                              /opt/altera/altera12.1/nios2eds/bin/gnu/H-i686-pc-linux-gnu/bin/../lib/gcc/nios2-elf/4.1.2/../../../../nios2-elf/lib/mno-hw-mul/libc.a(lib_a-exit.o) (_global_impure_ptr)
/opt/altera/altera12.1/nios2eds/bin/gnu/H-i686-pc-linux-gnu/bin/../lib/gcc/nios2-elf/4.1.2/../../../../nios2-elf/lib/mno-hw-mul/libc.a(lib_a-int_errno.o)
                              ../snake_software_bsp//libhal_bsp.a(alt_close.o) (errno)
/opt/altera/altera12.1/nios2eds/bin/gnu/H-i686-pc-linux-gnu/bin/../lib/gcc/nios2-elf/4.1.2/../../../../nios2-elf/lib/mno-hw-mul/libc.a(lib_a-memcmp.o)
                              ../snake_software_bsp//libhal_bsp.a(alt_find_dev.o) (memcmp)
/opt/altera/altera12.1/nios2eds/bin/gnu/H-i686-pc-linux-gnu/bin/../lib/gcc/nios2-elf/4.1.2/../../../../nios2-elf/lib/mno-hw-mul/libc.a(lib_a-memcpy.o)
                              ../snake_software_bsp//libhal_bsp.a(altera_avalon_jtag_uart_read.o) (memcpy)
/opt/altera/altera12.1/nios2eds/bin/gnu/H-i686-pc-linux-gnu/bin/../lib/gcc/nios2-elf/4.1.2/../../../../nios2-elf/lib/mno-hw-mul/libc.a(lib_a-strlen.o)
                              ../snake_software_bsp//libhal_bsp.a(alt_find_dev.o) (strlen)
/opt/altera/altera12.1/nios2eds/bin/gnu/H-i686-pc-linux-gnu/bin/../lib/gcc/nios2-elf/4.1.2/../../../../nios2-elf/lib/mno-hw-mul/libc.a(lib_a-__atexit.o)
                              /opt/altera/altera12.1/nios2eds/bin/gnu/H-i686-pc-linux-gnu/bin/../lib/gcc/nios2-elf/4.1.2/../../../../nios2-elf/lib/mno-hw-mul/libc.a(lib_a-atexit.o) (__register_exitproc)
/opt/altera/altera12.1/nios2eds/bin/gnu/H-i686-pc-linux-gnu/bin/../lib/gcc/nios2-elf/4.1.2/../../../../nios2-elf/lib/mno-hw-mul/libc.a(lib_a-__call_atexit.o)
                              /opt/altera/altera12.1/nios2eds/bin/gnu/H-i686-pc-linux-gnu/bin/../lib/gcc/nios2-elf/4.1.2/../../../../nios2-elf/lib/mno-hw-mul/libc.a(lib_a-exit.o) (__call_exitprocs)
../snake_software_bsp//libhal_bsp.a(alt_exit.o)
                              /opt/altera/altera12.1/nios2eds/bin/gnu/H-i686-pc-linux-gnu/bin/../lib/gcc/nios2-elf/4.1.2/../../../../nios2-elf/lib/mno-hw-mul/libc.a(lib_a-exit.o) (_exit)

Allocating common symbols
Common symbol       size              file

food                0x960             obj/default/main.o
alt_irq             0x100             ../snake_software_bsp//libhal_bsp.a(alt_irq_handler.o)
x                   0xa0              obj/default/main.o
PLAYER2_SLEEP_CYCLES
                    0x4               obj/default/main.o
errno               0x4               /opt/altera/altera12.1/nios2eds/bin/gnu/H-i686-pc-linux-gnu/bin/../lib/gcc/nios2-elf/4.1.2/../../../../nios2-elf/lib/mno-hw-mul/libc.a(lib_a-int_errno.o)
board               0x12c0            obj/default/main.o
PLAYER1_SLEEP_CYCLES
                    0x4               obj/default/main.o
brick_tiles         0x960             obj/default/main.o
edwards             0x960             obj/default/main.o
_atexit0            0x190             /opt/altera/altera12.1/nios2eds/bin/gnu/H-i686-pc-linux-gnu/bin/../lib/gcc/nios2-elf/4.1.2/../../../../nios2-elf/lib/mno-hw-mul/libc.a(lib_a-atexit.o)
y                   0x78              obj/default/main.o
speed               0x708             obj/default/main.o
freeze              0x708             obj/default/main.o

Memory Configuration

Name             Origin             Length             Attributes
reset            0x00080000         0x00000020
sram             0x00080020         0x0007ffe0
*default*        0x00000000         0xffffffff

Linker script and memory map

LOAD ../snake_software_bsp//obj/HAL/src/crt0.o
LOAD obj/default/hello_world.o
LOAD obj/default/main.o
LOAD /opt/altera/altera12.1/nios2eds/bin/gnu/H-i686-pc-linux-gnu/bin/../lib/gcc/nios2-elf/4.1.2/../../../../nios2-elf/lib/mno-hw-mul/libstdc++.a
LOAD /opt/altera/altera12.1/nios2eds/bin/gnu/H-i686-pc-linux-gnu/bin/../lib/gcc/nios2-elf/4.1.2/../../../../nios2-elf/lib/mno-hw-mul/libm.a
LOAD /opt/altera/altera12.1/nios2eds/bin/gnu/H-i686-pc-linux-gnu/bin/../lib/gcc/nios2-elf/4.1.2/mno-hw-mul/libgcc.a
START GROUP
LOAD /opt/altera/altera12.1/nios2eds/bin/gnu/H-i686-pc-linux-gnu/bin/../lib/gcc/nios2-elf/4.1.2/../../../../nios2-elf/lib/mno-hw-mul/libc.a
LOAD /opt/altera/altera12.1/nios2eds/bin/gnu/H-i686-pc-linux-gnu/bin/../lib/gcc/nios2-elf/4.1.2/mno-hw-mul/libgcc.a
LOAD ../snake_software_bsp//libhal_bsp.a
END GROUP
LOAD /opt/altera/altera12.1/nios2eds/bin/gnu/H-i686-pc-linux-gnu/bin/../lib/gcc/nios2-elf/4.1.2/mno-hw-mul/libgcc.a
                0x00080000                __alt_mem_sram = 0x80000

.entry          0x00080000       0x20
 *(.entry)
 .entry         0x00080000       0x20 ../snake_software_bsp//obj/HAL/src/crt0.o
                0x00080000                __reset

.exceptions     0x00080020      0x194
                0x00080020                PROVIDE (__ram_exceptions_start, ABSOLUTE (.))
                0x00080020                . = ALIGN (0x20)
 *(.irq)
 *(.exceptions.entry.label)
 .exceptions.entry.label
                0x00080020        0x0 ../snake_software_bsp//libhal_bsp.a(alt_irq_entry.o)
                0x00080020                alt_irq_entry
 .exceptions.entry.label
                0x00080020        0x0 ../snake_software_bsp//libhal_bsp.a(alt_exception_entry.o)
                0x00080020                alt_exception
 *(.exceptions.entry.user)
 *(.exceptions.entry)
 .exceptions.entry
                0x00080020       0x54 ../snake_software_bsp//libhal_bsp.a(alt_exception_entry.o)
 *(.exceptions.irqtest.user)
 *(.exceptions.irqtest)
 .exceptions.irqtest
                0x00080074       0x10 ../snake_software_bsp//libhal_bsp.a(alt_irq_entry.o)
 *(.exceptions.irqhandler.user)
 *(.exceptions.irqhandler)
 .exceptions.irqhandler
                0x00080084        0x4 ../snake_software_bsp//libhal_bsp.a(alt_irq_entry.o)
 *(.exceptions.irqreturn.user)
 *(.exceptions.irqreturn)
 .exceptions.irqreturn
                0x00080088        0x4 ../snake_software_bsp//libhal_bsp.a(alt_irq_entry.o)
 *(.exceptions.notirq.label)
 .exceptions.notirq.label
                0x0008008c        0x0 ../snake_software_bsp//libhal_bsp.a(alt_irq_entry.o)
 *(.exceptions.notirq.user)
 *(.exceptions.notirq)
 .exceptions.notirq
                0x0008008c        0x8 ../snake_software_bsp//libhal_bsp.a(alt_exception_entry.o)
 *(.exceptions.soft.user)
 *(.exceptions.soft)
 *(.exceptions.unknown.user)
 *(.exceptions.unknown)
 .exceptions.unknown
                0x00080094        0x4 ../snake_software_bsp//libhal_bsp.a(alt_exception_entry.o)
 *(.exceptions.exit.label)
 .exceptions.exit.label
                0x00080098        0x0 ../snake_software_bsp//libhal_bsp.a(alt_irq_entry.o)
 .exceptions.exit.label
                0x00080098        0x0 ../snake_software_bsp//libhal_bsp.a(alt_exception_entry.o)
 *(.exceptions.exit.user)
 *(.exceptions.exit)
 .exceptions.exit
                0x00080098       0x54 ../snake_software_bsp//libhal_bsp.a(alt_exception_entry.o)
 *(.exceptions)
 .exceptions    0x000800ec       0xc8 ../snake_software_bsp//libhal_bsp.a(alt_irq_handler.o)
                0x000800ec                alt_irq_handler
                0x000801b4                PROVIDE (__ram_exceptions_end, ABSOLUTE (.))
                0x00080020                PROVIDE (__flash_exceptions_start, LOADADDR (.exceptions))

.text           0x000801b4     0x8ce8
                0x000801b4                PROVIDE (stext, ABSOLUTE (.))
 *(.interp)
 *(.hash)
 *(.dynsym)
 *(.dynstr)
 *(.gnu.version)
 *(.gnu.version_d)
 *(.gnu.version_r)
 *(.rel.init)
 *(.rela.init)
 *(.rel.text .rel.text.* .rel.gnu.linkonce.t.*)
 *(.rela.text .rela.text.* .rela.gnu.linkonce.t.*)
 *(.rel.fini)
 *(.rela.fini)
 *(.rel.rodata .rel.rodata.* .rel.gnu.linkonce.r.*)
 *(.rela.rodata .rela.rodata.* .rela.gnu.linkonce.r.*)
 *(.rel.data .rel.data.* .rel.gnu.linkonce.d.*)
 *(.rela.data .rela.data.* .rela.gnu.linkonce.d.*)
 *(.rel.tdata .rel.tdata.* .rel.gnu.linkonce.td.*)
 *(.rela.tdata .rela.tdata.* .rela.gnu.linkonce.td.*)
 *(.rel.tbss .rel.tbss.* .rel.gnu.linkonce.tb.*)
 *(.rela.tbss .rela.tbss.* .rela.gnu.linkonce.tb.*)
 *(.rel.ctors)
 *(.rela.ctors)
 *(.rel.dtors)
 *(.rela.dtors)
 *(.rel.got)
 *(.rela.got)
 *(.rel.sdata .rel.sdata.* .rel.gnu.linkonce.s.*)
 *(.rela.sdata .rela.sdata.* .rela.gnu.linkonce.s.*)
 *(.rel.sbss .rel.sbss.* .rel.gnu.linkonce.sb.*)
 *(.rela.sbss .rela.sbss.* .rela.gnu.linkonce.sb.*)
 *(.rel.sdata2 .rel.sdata2.* .rel.gnu.linkonce.s2.*)
 *(.rela.sdata2 .rela.sdata2.* .rela.gnu.linkonce.s2.*)
 *(.rel.sbss2 .rel.sbss2.* .rel.gnu.linkonce.sb2.*)
 *(.rela.sbss2 .rela.sbss2.* .rela.gnu.linkonce.sb2.*)
 *(.rel.bss .rel.bss.* .rel.gnu.linkonce.b.*)
 *(.rela.bss .rela.bss.* .rela.gnu.linkonce.b.*)
 *(.rel.plt)
 *(.rela.plt)
 *(.rel.dyn)
 *(.init)
 *(.plt)
 *(.text .stub .text.* .gnu.linkonce.t.*)
 .text          0x000801b4       0x3c ../snake_software_bsp//obj/HAL/src/crt0.o
                0x000801b4                _start
 .text          0x000801f0        0x0 obj/default/hello_world.o
 .text          0x000801f0     0x6714 obj/default/main.o
                0x000801f0                addSnakePiece
                0x000802c8                removeSnakePiece
                0x000803a0                addTilePiece
                0x0008046c                removeTilePiece
                0x00080538                getController
                0x00080580                getPlayer1Controller
                0x000805c0                getPlayer2Controller
                0x00080600                get_dir_from_pressed
                0x000806c8                get_button_from_pressed
                0x00080744                check_paused
                0x00080770                enable_splash_screen
                0x00080798                disable_splash_screen
                0x000807c0                reset_hardware
                0x000808d4                PRNG
                0x0008092c                shuffle
                0x000809fc                shuffle2d
                0x00080b68                initPowBoard
                0x00080d18                initSnake
                0x00081008                abs
                0x00081044                traverseList
                0x00081180                brickCol
                0x00081250                snakeCol
                0x00081504                addEnd
                0x000818b4                updateBody
                0x00081998                updateSnake
                0x00081ce0                play_move_sound
                0x00081d18                play_powerup_sound
                0x00081d44                play_gameover_sound
                0x00081d70                play_splash_sound
                0x00081d9c                play_sound
                0x00081e0c                initFood
                0x00081f70                checkFood
                0x00082144                drawFood
                0x00082694                removeFood
                0x00082734                shuffle_food
                0x00082838                initSpeed
                0x00082964                checkSpeed
                0x00082be4                drawSpeed
                0x000830cc                removeSpeed
                0x00083184                shuffle_speed
                0x0008329c                initFreeze
                0x000833d0                checkFreeze
                0x00083568                apply_freeze
                0x0008360c                recalc_freeze_times
                0x000836dc                drawFreeze
                0x00083bc4                removeFreeze
                0x00083c70                shuffle_freeze
                0x00083d78                initBorder
                0x00083ec4                updateBorder
                0x00084190                checkOverlap
                0x00084574                initBrickTile
                0x000846d0                setBrickTile
                0x00084794                initEdwards
                0x0008493c                drawEdwards
                0x00084df4                removeEdwards
                0x00084e8c                shuffle_edwards
                0x00084f90                checkEdwards
                0x00085104                apply_edwards
                0x00085260                moveLeft
                0x000852b0                moveRight
                0x00085300                moveUp
                0x00085350                moveDown
                0x000853a0                movement
                0x000857ac                writeToHW
                0x00085a5c                check_powerup_col
                0x00085af8                check_powerup_buttons
                0x00085b74                wait_for_continue
                0x00085bd0                draw_P1_wins
                0x00085cc0                draw_P2_wins
                0x00085db4                draw_tie
                0x00085e50                draw_paused
                0x00085e98                draw_winner
                0x00085ff0                initPowUps
                0x00086024                drawStartPowUps
                0x000860c8                reset_software
                0x00086174                fancy_splash
                0x000864b0                main
 .text          0x00086904      0x14c /opt/altera/altera12.1/nios2eds/bin/gnu/H-i686-pc-linux-gnu/bin/../lib/gcc/nios2-elf/4.1.2/mno-hw-mul/libgcc.a(lib2-divmod.o)
                0x00086980                __divsi3
                0x000869e0                __modsi3
                0x00086a40                __udivsi3
                0x00086a48                __umodsi3
 .text          0x00086a50       0x38 /opt/altera/altera12.1/nios2eds/bin/gnu/H-i686-pc-linux-gnu/bin/../lib/gcc/nios2-elf/4.1.2/mno-hw-mul/libgcc.a(lib2-mul.o)
                0x00086a50                __mulsi3
 .text          0x00086a88       0xec ../snake_software_bsp//libhal_bsp.a(alt_load.o)
                0x00086a88                alt_load
 .text          0x00086b74       0x6c ../snake_software_bsp//libhal_bsp.a(alt_main.o)
                0x00086b74                alt_main
 .text          0x00086be0       0x30 ../snake_software_bsp//libhal_bsp.a(alt_usleep.o)
                0x00086be0                usleep
 .text          0x00086c10       0xb0 ../snake_software_bsp//libhal_bsp.a(alt_sys_init.o)
                0x00086c10                alt_irq_init
                0x00086c44                alt_sys_init
 .text          0x00086cc0      0x148 ../snake_software_bsp//libhal_bsp.a(altera_avalon_jtag_uart_fd.o)
                0x00086cc0                altera_avalon_jtag_uart_read_fd
                0x00086d18                altera_avalon_jtag_uart_write_fd
                0x00086d70                altera_avalon_jtag_uart_close_fd
                0x00086db8                altera_avalon_jtag_uart_ioctl_fd
 .text          0x00086e08      0x40c ../snake_software_bsp//libhal_bsp.a(altera_avalon_jtag_uart_init.o)
                0x00086e08                altera_avalon_jtag_uart_init
                0x000871a0                altera_avalon_jtag_uart_close
 .text          0x00087214       0xf4 ../snake_software_bsp//libhal_bsp.a(altera_avalon_jtag_uart_ioctl.o)
                0x00087214                altera_avalon_jtag_uart_ioctl
 .text          0x00087308      0x224 ../snake_software_bsp//libhal_bsp.a(altera_avalon_jtag_uart_read.o)
                0x00087308                altera_avalon_jtag_uart_read
 .text          0x0008752c      0x240 ../snake_software_bsp//libhal_bsp.a(altera_avalon_jtag_uart_write.o)
                0x0008752c                altera_avalon_jtag_uart_write
 .text          0x0008776c      0x154 ../snake_software_bsp//libhal_bsp.a(alt_alarm_start.o)
                0x0008776c                alt_alarm_start
 .text          0x000878c0      0x15c ../snake_software_bsp//libhal_bsp.a(alt_busy_sleep.o)
                0x000878c0                alt_busy_sleep
 .text          0x00087a1c      0x160 ../snake_software_bsp//libhal_bsp.a(alt_close.o)
                0x00087a1c                close
 .text          0x00087b7c       0x1c ../snake_software_bsp//libhal_bsp.a(alt_dcache_flush_all.o)
                0x00087b7c                alt_dcache_flush_all
 .text          0x00087b98       0x2c ../snake_software_bsp//libhal_bsp.a(alt_dev.o)
 .text          0x00087bc4      0x114 ../snake_software_bsp//libhal_bsp.a(alt_dev_llist_insert.o)
                0x00087bc4                alt_dev_llist_insert
 .text          0x00087cd8       0x64 ../snake_software_bsp//libhal_bsp.a(alt_do_ctors.o)
                0x00087cd8                _do_ctors
 .text          0x00087d3c       0x64 ../snake_software_bsp//libhal_bsp.a(alt_do_dtors.o)
                0x00087d3c                _do_dtors
 .text          0x00087da0        0x0 ../snake_software_bsp//libhal_bsp.a(alt_errno.o)
 .text          0x00087da0       0x1c ../snake_software_bsp//libhal_bsp.a(alt_icache_flush_all.o)
                0x00087da0                alt_icache_flush_all
 .text          0x00087dbc      0x1d4 ../snake_software_bsp//libhal_bsp.a(alt_iic.o)
                0x00087dbc                alt_ic_isr_register
                0x00087e0c                alt_ic_irq_enable
                0x00087ea8                alt_ic_irq_disable
                0x00087f48                alt_ic_irq_enabled
 .text          0x00087f90       0xf8 ../snake_software_bsp//libhal_bsp.a(alt_iic_isr_register.o)
                0x00087f90                alt_iic_isr_register
 .text          0x00088088      0x150 ../snake_software_bsp//libhal_bsp.a(alt_io_redirect.o)
                0x00088160                alt_io_redirect
 .text          0x000881d8        0x0 ../snake_software_bsp//libhal_bsp.a(alt_irq_entry.o)
 .text          0x000881d8        0x0 ../snake_software_bsp//libhal_bsp.a(alt_irq_handler.o)
 .text          0x000881d8        0x0 ../snake_software_bsp//libhal_bsp.a(alt_irq_vars.o)
 .text          0x000881d8      0x2e4 ../snake_software_bsp//libhal_bsp.a(alt_open.o)
                0x000882d0                open
 .text          0x000884bc       0x78 ../snake_software_bsp//libhal_bsp.a(alt_release_fd.o)
                0x000884bc                alt_release_fd
 .text          0x00088534      0x1a4 ../snake_software_bsp//libhal_bsp.a(alt_tick.o)
                0x00088534                alt_alarm_stop
                0x000885cc                alt_tick
 .text          0x000886d8       0x20 ../snake_software_bsp//libhal_bsp.a(altera_nios2_irq.o)
                0x000886d8                altera_nios2_irq_init
 .text          0x000886f8        0x0 ../snake_software_bsp//libhal_bsp.a(alt_exception_entry.o)
 .text          0x000886f8       0x94 ../snake_software_bsp//libhal_bsp.a(alt_find_dev.o)
                0x000886f8                alt_find_dev
 .text          0x0008878c      0x120 ../snake_software_bsp//libhal_bsp.a(alt_find_file.o)
                0x0008878c                alt_find_file
 .text          0x000888ac       0xd0 ../snake_software_bsp//libhal_bsp.a(alt_get_fd.o)
                0x000888ac                alt_get_fd
 .text          0x0008897c       0x14 /opt/altera/altera12.1/nios2eds/bin/gnu/H-i686-pc-linux-gnu/bin/../lib/gcc/nios2-elf/4.1.2/../../../../nios2-elf/lib/mno-hw-mul/libc.a(lib_a-atexit.o)
                0x0008897c                atexit
 .text          0x00088990       0x38 /opt/altera/altera12.1/nios2eds/bin/gnu/H-i686-pc-linux-gnu/bin/../lib/gcc/nios2-elf/4.1.2/../../../../nios2-elf/lib/mno-hw-mul/libc.a(lib_a-exit.o)
                0x00088990                exit
 .text          0x000889c8        0x0 /opt/altera/altera12.1/nios2eds/bin/gnu/H-i686-pc-linux-gnu/bin/../lib/gcc/nios2-elf/4.1.2/../../../../nios2-elf/lib/mno-hw-mul/libc.a(lib_a-impure.o)
 .text          0x000889c8        0x0 /opt/altera/altera12.1/nios2eds/bin/gnu/H-i686-pc-linux-gnu/bin/../lib/gcc/nios2-elf/4.1.2/../../../../nios2-elf/lib/mno-hw-mul/libc.a(lib_a-int_errno.o)
 .text          0x000889c8       0x74 /opt/altera/altera12.1/nios2eds/bin/gnu/H-i686-pc-linux-gnu/bin/../lib/gcc/nios2-elf/4.1.2/../../../../nios2-elf/lib/mno-hw-mul/libc.a(lib_a-memcmp.o)
                0x000889c8                memcmp
 .text          0x00088a3c       0xa0 /opt/altera/altera12.1/nios2eds/bin/gnu/H-i686-pc-linux-gnu/bin/../lib/gcc/nios2-elf/4.1.2/../../../../nios2-elf/lib/mno-hw-mul/libc.a(lib_a-memcpy.o)
                0x00088a3c                memcpy
 .text          0x00088adc       0x74 /opt/altera/altera12.1/nios2eds/bin/gnu/H-i686-pc-linux-gnu/bin/../lib/gcc/nios2-elf/4.1.2/../../../../nios2-elf/lib/mno-hw-mul/libc.a(lib_a-strlen.o)
                0x00088adc                strlen
 .text          0x00088b50      0x134 /opt/altera/altera12.1/nios2eds/bin/gnu/H-i686-pc-linux-gnu/bin/../lib/gcc/nios2-elf/4.1.2/../../../../nios2-elf/lib/mno-hw-mul/libc.a(lib_a-__atexit.o)
                0x00088b50                __register_exitproc
 .text          0x00088c84      0x1b4 /opt/altera/altera12.1/nios2eds/bin/gnu/H-i686-pc-linux-gnu/bin/../lib/gcc/nios2-elf/4.1.2/../../../../nios2-elf/lib/mno-hw-mul/libc.a(lib_a-__call_atexit.o)
                0x00088c88                __call_exitprocs
 .text          0x00088e38       0x60 ../snake_software_bsp//libhal_bsp.a(alt_exit.o)
                0x00088e78                _exit
 *(.gnu.warning.*)
 *(.fini)
                0x00088e98                PROVIDE (__etext, ABSOLUTE (.))
                0x00088e98                PROVIDE (_etext, ABSOLUTE (.))
                0x00088e98                PROVIDE (etext, ABSOLUTE (.))
 *(.eh_frame_hdr)
                0x00088e98                . = ALIGN (0x4)
                0x00088e98                PROVIDE (__preinit_array_start, ABSOLUTE (.))
 *(.preinit_array)
                0x00088e98                PROVIDE (__preinit_array_end, ABSOLUTE (.))
                0x00088e98                PROVIDE (__init_array_start, ABSOLUTE (.))
 *(.init_array)
                0x00088e98                PROVIDE (__init_array_end, ABSOLUTE (.))
                0x00088e98                PROVIDE (__fini_array_start, ABSOLUTE (.))
 *(.fini_array)
                0x00088e98                PROVIDE (__fini_array_end, ABSOLUTE (.))
 *(.eh_frame)
 *(.gcc_except_table)
 *(.dynamic)
                0x00088e98                PROVIDE (__CTOR_LIST__, ABSOLUTE (.))
 *(.ctors)
 *(SORT(.ctors.*))
 .ctors.65535   0x00088e98        0x4 /opt/altera/altera12.1/nios2eds/bin/gnu/H-i686-pc-linux-gnu/bin/../lib/gcc/nios2-elf/4.1.2/../../../../nios2-elf/lib/mno-hw-mul/libc.a(lib_a-__call_atexit.o)
                0x00088e9c                PROVIDE (__CTOR_END__, ABSOLUTE (.))
                0x00088e9c                PROVIDE (__DTOR_LIST__, ABSOLUTE (.))
 *(.dtors)
 *(SORT(.dtors.*))
                0x00088e9c                PROVIDE (__DTOR_END__, ABSOLUTE (.))
 *(.jcr)
                0x00088e9c                . = ALIGN (0x4)

.rodata         0x00088e9c       0x38
                0x00088e9c                PROVIDE (__ram_rodata_start, ABSOLUTE (.))
                0x00088e9c                . = ALIGN (0x4)
 *(.rodata .rodata.* .gnu.linkonce.r.*)
 .rodata        0x00088e9c       0x14 ../snake_software_bsp//libhal_bsp.a(alt_main.o)
 .rodata        0x00088eb0       0x14 ../snake_software_bsp//libhal_bsp.a(alt_sys_init.o)
 .rodata        0x00088ec4        0xc ../snake_software_bsp//libhal_bsp.a(alt_dev.o)
 .rodata.str1.4
                0x00088ed0        0x4 /opt/altera/altera12.1/nios2eds/bin/gnu/H-i686-pc-linux-gnu/bin/../lib/gcc/nios2-elf/4.1.2/../../../../nios2-elf/lib/mno-hw-mul/libc.a(lib_a-impure.o)
 *(.rodata1)
                0x00088ed4                . = ALIGN (0x4)
                0x00088ed4                PROVIDE (__ram_rodata_end, ABSOLUTE (.))
                0x00088e9c                PROVIDE (__flash_rodata_start, LOADADDR (.rodata))

.rwdata         0x00088ed4     0x16e0 load address 0x0008a5b4
                0x00088ed4                PROVIDE (__ram_rwdata_start, ABSOLUTE (.))
                0x00088ed4                . = ALIGN (0x4)
 *(.got.plt)
 *(.got)
 *(.data1)
 *(.data .data.* .gnu.linkonce.d.*)
 .data          0x00088ed4        0x0 ../snake_software_bsp//obj/HAL/src/crt0.o
 .data          0x00088ed4        0x0 obj/default/hello_world.o
 .data          0x00088ed4        0x0 obj/default/main.o
 .data          0x00088ed4        0x0 /opt/altera/altera12.1/nios2eds/bin/gnu/H-i686-pc-linux-gnu/bin/../lib/gcc/nios2-elf/4.1.2/mno-hw-mul/libgcc.a(lib2-divmod.o)
 .data          0x00088ed4        0x0 /opt/altera/altera12.1/nios2eds/bin/gnu/H-i686-pc-linux-gnu/bin/../lib/gcc/nios2-elf/4.1.2/mno-hw-mul/libgcc.a(lib2-mul.o)
 .data          0x00088ed4        0x0 ../snake_software_bsp//libhal_bsp.a(alt_load.o)
 .data          0x00088ed4        0x0 ../snake_software_bsp//libhal_bsp.a(alt_main.o)
 .data          0x00088ed4        0x0 ../snake_software_bsp//libhal_bsp.a(alt_usleep.o)
 .data          0x00088ed4     0x1060 ../snake_software_bsp//libhal_bsp.a(alt_sys_init.o)
 .data          0x00089f34        0x0 ../snake_software_bsp//libhal_bsp.a(altera_avalon_jtag_uart_fd.o)
 .data          0x00089f34        0x0 ../snake_software_bsp//libhal_bsp.a(altera_avalon_jtag_uart_init.o)
 .data          0x00089f34        0x0 ../snake_software_bsp//libhal_bsp.a(altera_avalon_jtag_uart_ioctl.o)
 .data          0x00089f34        0x0 ../snake_software_bsp//libhal_bsp.a(altera_avalon_jtag_uart_read.o)
 .data          0x00089f34        0x0 ../snake_software_bsp//libhal_bsp.a(altera_avalon_jtag_uart_write.o)
 .data          0x00089f34        0x0 ../snake_software_bsp//libhal_bsp.a(alt_alarm_start.o)
 .data          0x00089f34        0x0 ../snake_software_bsp//libhal_bsp.a(alt_busy_sleep.o)
 .data          0x00089f34        0x0 ../snake_software_bsp//libhal_bsp.a(alt_close.o)
 .data          0x00089f34        0x0 ../snake_software_bsp//libhal_bsp.a(alt_dcache_flush_all.o)
 .data          0x00089f34      0x1a8 ../snake_software_bsp//libhal_bsp.a(alt_dev.o)
                0x00089f34                alt_dev_null
                0x00089f5c                alt_fd_list
 .data          0x0008a0dc        0x0 ../snake_software_bsp//libhal_bsp.a(alt_dev_llist_insert.o)
 .data          0x0008a0dc        0x0 ../snake_software_bsp//libhal_bsp.a(alt_do_ctors.o)
 .data          0x0008a0dc        0x0 ../snake_software_bsp//libhal_bsp.a(alt_do_dtors.o)
 .data          0x0008a0dc        0x0 ../snake_software_bsp//libhal_bsp.a(alt_errno.o)
 .data          0x0008a0dc        0x0 ../snake_software_bsp//libhal_bsp.a(alt_icache_flush_all.o)
 .data          0x0008a0dc        0x0 ../snake_software_bsp//libhal_bsp.a(alt_iic.o)
 .data          0x0008a0dc        0x0 ../snake_software_bsp//libhal_bsp.a(alt_iic_isr_register.o)
 .data          0x0008a0dc        0x0 ../snake_software_bsp//libhal_bsp.a(alt_io_redirect.o)
 .data          0x0008a0dc        0x0 ../snake_software_bsp//libhal_bsp.a(alt_irq_entry.o)
 .data          0x0008a0dc        0x0 ../snake_software_bsp//libhal_bsp.a(alt_irq_handler.o)
 .data          0x0008a0dc        0x0 ../snake_software_bsp//libhal_bsp.a(alt_irq_vars.o)
 .data          0x0008a0dc        0x0 ../snake_software_bsp//libhal_bsp.a(alt_open.o)
 .data          0x0008a0dc        0x0 ../snake_software_bsp//libhal_bsp.a(alt_release_fd.o)
 .data          0x0008a0dc        0x0 ../snake_software_bsp//libhal_bsp.a(alt_tick.o)
 .data          0x0008a0dc        0x0 ../snake_software_bsp//libhal_bsp.a(altera_nios2_irq.o)
 .data          0x0008a0dc        0x0 ../snake_software_bsp//libhal_bsp.a(alt_exception_entry.o)
 .data          0x0008a0dc        0x0 ../snake_software_bsp//libhal_bsp.a(alt_find_dev.o)
 .data          0x0008a0dc        0x0 ../snake_software_bsp//libhal_bsp.a(alt_find_file.o)
 .data          0x0008a0dc        0x0 ../snake_software_bsp//libhal_bsp.a(alt_get_fd.o)
 .data          0x0008a0dc        0x0 /opt/altera/altera12.1/nios2eds/bin/gnu/H-i686-pc-linux-gnu/bin/../lib/gcc/nios2-elf/4.1.2/../../../../nios2-elf/lib/mno-hw-mul/libc.a(lib_a-atexit.o)
 .data          0x0008a0dc        0x0 /opt/altera/altera12.1/nios2eds/bin/gnu/H-i686-pc-linux-gnu/bin/../lib/gcc/nios2-elf/4.1.2/../../../../nios2-elf/lib/mno-hw-mul/libc.a(lib_a-exit.o)
 .data          0x0008a0dc      0x400 /opt/altera/altera12.1/nios2eds/bin/gnu/H-i686-pc-linux-gnu/bin/../lib/gcc/nios2-elf/4.1.2/../../../../nios2-elf/lib/mno-hw-mul/libc.a(lib_a-impure.o)
 .data          0x0008a4dc        0x0 /opt/altera/altera12.1/nios2eds/bin/gnu/H-i686-pc-linux-gnu/bin/../lib/gcc/nios2-elf/4.1.2/../../../../nios2-elf/lib/mno-hw-mul/libc.a(lib_a-int_errno.o)
 .data          0x0008a4dc        0x0 /opt/altera/altera12.1/nios2eds/bin/gnu/H-i686-pc-linux-gnu/bin/../lib/gcc/nios2-elf/4.1.2/../../../../nios2-elf/lib/mno-hw-mul/libc.a(lib_a-memcmp.o)
 .data          0x0008a4dc        0x0 /opt/altera/altera12.1/nios2eds/bin/gnu/H-i686-pc-linux-gnu/bin/../lib/gcc/nios2-elf/4.1.2/../../../../nios2-elf/lib/mno-hw-mul/libc.a(lib_a-memcpy.o)
 .data          0x0008a4dc        0x0 /opt/altera/altera12.1/nios2eds/bin/gnu/H-i686-pc-linux-gnu/bin/../lib/gcc/nios2-elf/4.1.2/../../../../nios2-elf/lib/mno-hw-mul/libc.a(lib_a-strlen.o)
 .data          0x0008a4dc        0x0 /opt/altera/altera12.1/nios2eds/bin/gnu/H-i686-pc-linux-gnu/bin/../lib/gcc/nios2-elf/4.1.2/../../../../nios2-elf/lib/mno-hw-mul/libc.a(lib_a-__atexit.o)
 .data          0x0008a4dc        0x0 /opt/altera/altera12.1/nios2eds/bin/gnu/H-i686-pc-linux-gnu/bin/../lib/gcc/nios2-elf/4.1.2/../../../../nios2-elf/lib/mno-hw-mul/libc.a(lib_a-__call_atexit.o)
 .data          0x0008a4dc        0x0 ../snake_software_bsp//libhal_bsp.a(alt_exit.o)
                0x000924dc                _gp = ABSOLUTE ((. + 0x8000))
                0x000924dc                PROVIDE (gp, _gp)
 *(.rwdata .rwdata.*)
 *(.sdata .sdata.* .gnu.linkonce.s.*)
 .sdata         0x0008a4dc       0xac obj/default/main.o
                0x0008a4dc                SNAKE_ADDR
                0x0008a4dd                TILES_ADDR
                0x0008a4de                PLAYER1
                0x0008a4df                PLAYER2
                0x0008a4e0                SNAKE_HEAD_RIGHT
                0x0008a4e1                SNAKE_HEAD_LEFT
                0x0008a4e2                SNAKE_HEAD_UP
                0x0008a4e3                SNAKE_HEAD_DOWN
                0x0008a4e4                SNAKE_TAIL_RIGHT
                0x0008a4e5                SNAKE_TAIL_LEFT
                0x0008a4e6                SNAKE_TAIL_UP
                0x0008a4e7                SNAKE_TAIL_DOWN
                0x0008a4e8                SNAKE_BODY_RIGHT
                0x0008a4e9                SNAKE_BODY_LEFT
                0x0008a4ea                SNAKE_BODY_UP
                0x0008a4eb                SNAKE_BODY_DOWN
                0x0008a4ec                SNAKE_TURN_UP_RIGHT
                0x0008a4ed                SNAKE_TURN_RIGHT_DOWN
                0x0008a4ee                SNAKE_TURN_DOWN_LEFT
                0x0008a4ef                SNAKE_TURN_LEFT_UP
                0x0008a4f0                RABBIT_CODE
                0x0008a4f1                MOUSE_CODE
                0x0008a4f2                EDWARDS_CODE
                0x0008a4f3                WALL_CODE
                0x0008a4f4                SPEED_CODE
                0x0008a4f5                FREEZE_CODE
                0x0008a4f6                GROWTH_CODE
                0x0008a4f7                ONE_CODE
                0x0008a4f8                TWO_CODE
                0x0008a4f9                P_CODE
                0x0008a4fa                W_CODE
                0x0008a4fb                I_CODE
                0x0008a4fc                N_CODE
                0x0008a4fd                S_CODE
                0x0008a4fe                EXC_CODE
                0x0008a4ff                PLAY_CODE
                0x0008a500                PAUSE_CODE
                0x0008a501                SPLASH_SNAKE_CODE
                0x0008a502                T_CODE
                0x0008a503                E_CODE
                0x0008a504                SEG_HEAD
                0x0008a505                SEG_SECOND_HEAD
                0x0008a506                SEG_SECOND_TAIL
                0x0008a507                SEG_TAIL
                0x0008a508                REMOVE_CODE
                0x0008a509                ADD_CODE
                0x0008a50c                RIGHT_CODE
                0x0008a510                LEFT_CODE
                0x0008a514                DOWN_CODE
                0x0008a518                UP_CODE
                0x0008a51c                START_CODE
                0x0008a520                SELECT_CODE
                0x0008a524                B_CODE
                0x0008a528                A_CODE
                0x0008a52c                DEFAULT_SLEEP_CYCLE
                0x0008a530                SPEED_SLEEP_CYCLE
                0x0008a534                FREEZE_SLEEP_CYCLE
                0x0008a538                n_seed
                0x0008a53c                food_index
                0x0008a540                speed_index
                0x0008a544                freeze_index
                0x0008a548                edwards_index
                0x0008a54c                RIGHT_BOUND
                0x0008a550                BOT_BOUND
                0x0008a554                NEW_BOT
                0x0008a558                NEW_RIGHT
                0x0008a55c                offset
                0x0008a560                sound_to_be_played
                0x0008a564                sound_divider
                0x0008a568                move_sound_code
                0x0008a56c                move_sound_divider
                0x0008a570                powerup_sound_code
                0x0008a574                powerup_sound_divider
                0x0008a578                gameover_sound_code
                0x0008a57c                gameover_sound_divider
                0x0008a580                splash_sound_code
                0x0008a584                splash_sound_divider
 .sdata         0x0008a588       0x14 ../snake_software_bsp//libhal_bsp.a(alt_dev.o)
                0x0008a588                alt_fs_list
                0x0008a590                alt_dev_list
                0x0008a598                alt_max_fd
 .sdata         0x0008a59c        0x4 ../snake_software_bsp//libhal_bsp.a(alt_errno.o)
                0x0008a59c                alt_errno
 .sdata         0x0008a5a0        0x4 ../snake_software_bsp//libhal_bsp.a(alt_irq_vars.o)
                0x0008a5a0                alt_priority_mask
 .sdata         0x0008a5a4        0x8 ../snake_software_bsp//libhal_bsp.a(alt_tick.o)
                0x0008a5a4                alt_alarm_list
 .sdata         0x0008a5ac        0x8 /opt/altera/altera12.1/nios2eds/bin/gnu/H-i686-pc-linux-gnu/bin/../lib/gcc/nios2-elf/4.1.2/../../../../nios2-elf/lib/mno-hw-mul/libc.a(lib_a-impure.o)
                0x0008a5ac                _impure_ptr
                0x0008a5b0                _global_impure_ptr
 *(.sdata2 .sdata2.* .gnu.linkonce.s2.*)
                0x0008a5b4                . = ALIGN (0x4)
                0x0008a5b4                _edata = ABSOLUTE (.)
                0x0008a5b4                PROVIDE (edata, ABSOLUTE (.))
                0x0008a5b4                PROVIDE (__ram_rwdata_end, ABSOLUTE (.))
                0x0008a5b4                PROVIDE (__flash_rwdata_start, LOADADDR (.rwdata))

.bss            0x0008bc94     0x4104
                0x0008bc94                __bss_start = ABSOLUTE (.)
                0x0008bc94                PROVIDE (__sbss_start, ABSOLUTE (.))
                0x0008bc94                PROVIDE (___sbss_start, ABSOLUTE (.))
 *(.dynsbss)
 *(.sbss .sbss.* .gnu.linkonce.sb.*)
 .sbss          0x0008bc94       0x48 obj/default/main.o
                0x0008bc94                seed
                0x0008bc98                alt_powups
                0x0008bc9c                freeze_pow_count
                0x0008bca0                freeze_drawn
                0x0008bca4                speed_pow_count
                0x0008bca8                speed_drawn
                0x0008bcac                edwards_pow_count
                0x0008bcb0                edwards_drawn
                0x0008bcb4                dir_arg
                0x0008bcb8                switch_snakes
                0x0008bcbc                food_count
                0x0008bcc0                player1_food_eaten
                0x0008bcc4                player2_food_eaten
                0x0008bcc8                LEFT_BOUND
                0x0008bccc                TOP_BOUND
                0x0008bcd0                NEW_TOP
                0x0008bcd4                NEW_LEFT
                0x0008bcd8                game_winner
 .sbss          0x0008bcdc        0x8 obj/default/main.o
                0x0008bcdc                PLAYER2_SLEEP_CYCLES
                0x0008bce0                PLAYER1_SLEEP_CYCLES
 .sbss          0x0008bce4        0xc ../snake_software_bsp//libhal_bsp.a(alt_main.o)
                0x0008bce4                alt_argc
                0x0008bce8                alt_argv
                0x0008bcec                alt_envp
 .sbss          0x0008bcf0        0x4 ../snake_software_bsp//libhal_bsp.a(alt_irq_vars.o)
                0x0008bcf0                alt_irq_active
 .sbss          0x0008bcf4        0x8 ../snake_software_bsp//libhal_bsp.a(alt_tick.o)
                0x0008bcf4                _alt_tick_rate
                0x0008bcf8                _alt_nticks
 .sbss          0x0008bcfc        0x4 /opt/altera/altera12.1/nios2eds/bin/gnu/H-i686-pc-linux-gnu/bin/../lib/gcc/nios2-elf/4.1.2/../../../../nios2-elf/lib/mno-hw-mul/libc.a(lib_a-int_errno.o)
                0x0008bcfc                errno
 *(.sbss2 .sbss2.* .gnu.linkonce.sb2.*)
 *(.scommon)
                0x0008bd00                PROVIDE (__sbss_end, ABSOLUTE (.))
                0x0008bd00                PROVIDE (___sbss_end, ABSOLUTE (.))
 *(.dynbss)
 *(.bss .bss.* .gnu.linkonce.b.*)
 .bss           0x0008bd00        0x0 ../snake_software_bsp//obj/HAL/src/crt0.o
 .bss           0x0008bd00        0x0 obj/default/hello_world.o
 .bss           0x0008bd00        0x0 obj/default/main.o
 .bss           0x0008bd00        0x0 /opt/altera/altera12.1/nios2eds/bin/gnu/H-i686-pc-linux-gnu/bin/../lib/gcc/nios2-elf/4.1.2/mno-hw-mul/libgcc.a(lib2-divmod.o)
 .bss           0x0008bd00        0x0 /opt/altera/altera12.1/nios2eds/bin/gnu/H-i686-pc-linux-gnu/bin/../lib/gcc/nios2-elf/4.1.2/mno-hw-mul/libgcc.a(lib2-mul.o)
 .bss           0x0008bd00        0x0 ../snake_software_bsp//libhal_bsp.a(alt_load.o)
 .bss           0x0008bd00        0x0 ../snake_software_bsp//libhal_bsp.a(alt_main.o)
 .bss           0x0008bd00        0x0 ../snake_software_bsp//libhal_bsp.a(alt_usleep.o)
 .bss           0x0008bd00        0x0 ../snake_software_bsp//libhal_bsp.a(alt_sys_init.o)
 .bss           0x0008bd00        0x0 ../snake_software_bsp//libhal_bsp.a(altera_avalon_jtag_uart_fd.o)
 .bss           0x0008bd00        0x0 ../snake_software_bsp//libhal_bsp.a(altera_avalon_jtag_uart_init.o)
 .bss           0x0008bd00        0x0 ../snake_software_bsp//libhal_bsp.a(altera_avalon_jtag_uart_ioctl.o)
 .bss           0x0008bd00        0x0 ../snake_software_bsp//libhal_bsp.a(altera_avalon_jtag_uart_read.o)
 .bss           0x0008bd00        0x0 ../snake_software_bsp//libhal_bsp.a(altera_avalon_jtag_uart_write.o)
 .bss           0x0008bd00        0x0 ../snake_software_bsp//libhal_bsp.a(alt_alarm_start.o)
 .bss           0x0008bd00        0x0 ../snake_software_bsp//libhal_bsp.a(alt_busy_sleep.o)
 .bss           0x0008bd00        0x0 ../snake_software_bsp//libhal_bsp.a(alt_close.o)
 .bss           0x0008bd00        0x0 ../snake_software_bsp//libhal_bsp.a(alt_dcache_flush_all.o)
 .bss           0x0008bd00        0x0 ../snake_software_bsp//libhal_bsp.a(alt_dev.o)
 .bss           0x0008bd00        0x0 ../snake_software_bsp//libhal_bsp.a(alt_dev_llist_insert.o)
 .bss           0x0008bd00        0x0 ../snake_software_bsp//libhal_bsp.a(alt_do_ctors.o)
 .bss           0x0008bd00        0x0 ../snake_software_bsp//libhal_bsp.a(alt_do_dtors.o)
 .bss           0x0008bd00        0x0 ../snake_software_bsp//libhal_bsp.a(alt_errno.o)
 .bss           0x0008bd00        0x0 ../snake_software_bsp//libhal_bsp.a(alt_icache_flush_all.o)
 .bss           0x0008bd00        0x0 ../snake_software_bsp//libhal_bsp.a(alt_iic.o)
 .bss           0x0008bd00        0x0 ../snake_software_bsp//libhal_bsp.a(alt_iic_isr_register.o)
 .bss           0x0008bd00        0x0 ../snake_software_bsp//libhal_bsp.a(alt_io_redirect.o)
 .bss           0x0008bd00        0x0 ../snake_software_bsp//libhal_bsp.a(alt_irq_entry.o)
 .bss           0x0008bd00        0x0 ../snake_software_bsp//libhal_bsp.a(alt_irq_handler.o)
 .bss           0x0008bd00        0x0 ../snake_software_bsp//libhal_bsp.a(alt_irq_vars.o)
 .bss           0x0008bd00        0x0 ../snake_software_bsp//libhal_bsp.a(alt_open.o)
 .bss           0x0008bd00        0x0 ../snake_software_bsp//libhal_bsp.a(alt_release_fd.o)
 .bss           0x0008bd00        0x0 ../snake_software_bsp//libhal_bsp.a(alt_tick.o)
 .bss           0x0008bd00        0x0 ../snake_software_bsp//libhal_bsp.a(altera_nios2_irq.o)
 .bss           0x0008bd00        0x0 ../snake_software_bsp//libhal_bsp.a(alt_exception_entry.o)
 .bss           0x0008bd00        0x0 ../snake_software_bsp//libhal_bsp.a(alt_find_dev.o)
 .bss           0x0008bd00        0x0 ../snake_software_bsp//libhal_bsp.a(alt_find_file.o)
 .bss           0x0008bd00        0x0 ../snake_software_bsp//libhal_bsp.a(alt_get_fd.o)
 .bss           0x0008bd00        0x0 /opt/altera/altera12.1/nios2eds/bin/gnu/H-i686-pc-linux-gnu/bin/../lib/gcc/nios2-elf/4.1.2/../../../../nios2-elf/lib/mno-hw-mul/libc.a(lib_a-atexit.o)
 .bss           0x0008bd00        0x0 /opt/altera/altera12.1/nios2eds/bin/gnu/H-i686-pc-linux-gnu/bin/../lib/gcc/nios2-elf/4.1.2/../../../../nios2-elf/lib/mno-hw-mul/libc.a(lib_a-exit.o)
 .bss           0x0008bd00        0x0 /opt/altera/altera12.1/nios2eds/bin/gnu/H-i686-pc-linux-gnu/bin/../lib/gcc/nios2-elf/4.1.2/../../../../nios2-elf/lib/mno-hw-mul/libc.a(lib_a-impure.o)
 .bss           0x0008bd00        0x0 /opt/altera/altera12.1/nios2eds/bin/gnu/H-i686-pc-linux-gnu/bin/../lib/gcc/nios2-elf/4.1.2/../../../../nios2-elf/lib/mno-hw-mul/libc.a(lib_a-int_errno.o)
 .bss           0x0008bd00        0x0 /opt/altera/altera12.1/nios2eds/bin/gnu/H-i686-pc-linux-gnu/bin/../lib/gcc/nios2-elf/4.1.2/../../../../nios2-elf/lib/mno-hw-mul/libc.a(lib_a-memcmp.o)
 .bss           0x0008bd00        0x0 /opt/altera/altera12.1/nios2eds/bin/gnu/H-i686-pc-linux-gnu/bin/../lib/gcc/nios2-elf/4.1.2/../../../../nios2-elf/lib/mno-hw-mul/libc.a(lib_a-memcpy.o)
 .bss           0x0008bd00        0x0 /opt/altera/altera12.1/nios2eds/bin/gnu/H-i686-pc-linux-gnu/bin/../lib/gcc/nios2-elf/4.1.2/../../../../nios2-elf/lib/mno-hw-mul/libc.a(lib_a-strlen.o)
 .bss           0x0008bd00        0x0 /opt/altera/altera12.1/nios2eds/bin/gnu/H-i686-pc-linux-gnu/bin/../lib/gcc/nios2-elf/4.1.2/../../../../nios2-elf/lib/mno-hw-mul/libc.a(lib_a-__atexit.o)
 .bss           0x0008bd00        0x0 /opt/altera/altera12.1/nios2eds/bin/gnu/H-i686-pc-linux-gnu/bin/../lib/gcc/nios2-elf/4.1.2/../../../../nios2-elf/lib/mno-hw-mul/libc.a(lib_a-__call_atexit.o)
 .bss           0x0008bd00        0x0 ../snake_software_bsp//libhal_bsp.a(alt_exit.o)
 *(COMMON)
 COMMON         0x0008bd00     0x3e08 obj/default/main.o
                0x0008bd00                food
                0x0008c660                x
                0x0008c700                board
                0x0008d9c0                brick_tiles
                0x0008e320                edwards
                0x0008ec80                y
                0x0008ecf8                speed
                0x0008f400                freeze
 COMMON         0x0008fb08      0x100 ../snake_software_bsp//libhal_bsp.a(alt_irq_handler.o)
                0x0008fb08                alt_irq
 COMMON         0x0008fc08      0x190 /opt/altera/altera12.1/nios2eds/bin/gnu/H-i686-pc-linux-gnu/bin/../lib/gcc/nios2-elf/4.1.2/../../../../nios2-elf/lib/mno-hw-mul/libc.a(lib_a-atexit.o)
                0x0008fc08                _atexit0
                0x0008fd98                . = ALIGN (0x4)
                0x0008fd98                __bss_end = ABSOLUTE (.)

.sram           0x0008fd98        0x0
                0x0008fd98                PROVIDE (_alt_partition_sram_start, ABSOLUTE (.))
 *(.sram. sram.*)
                0x0008fd98                . = ALIGN (0x4)
                0x0008fd98                PROVIDE (_alt_partition_sram_end, ABSOLUTE (.))
                0x0008fd98                _end = ABSOLUTE (.)
                0x0008fd98                end = ABSOLUTE (.)
                0x0008fd98                __alt_stack_base = ABSOLUTE (.)
                0x0008fd98                PROVIDE (_alt_partition_sram_load_addr, LOADADDR (.sram))

.stab
 *(.stab)

.stabstr
 *(.stabstr)

.stab.excl
 *(.stab.excl)

.stab.exclstr
 *(.stab.exclstr)

.stab.index
 *(.stab.index)

.stab.indexstr
 *(.stab.indexstr)

.comment        0x00000000       0x23
 *(.comment)
 .comment       0x00000000       0x23 obj/default/hello_world.o
                                 0x24 (size before relaxing)
 .comment       0x00000000       0x24 obj/default/main.o
 .comment       0x00000000       0x24 /opt/altera/altera12.1/nios2eds/bin/gnu/H-i686-pc-linux-gnu/bin/../lib/gcc/nios2-elf/4.1.2/mno-hw-mul/libgcc.a(lib2-divmod.o)
 .comment       0x00000000       0x24 /opt/altera/altera12.1/nios2eds/bin/gnu/H-i686-pc-linux-gnu/bin/../lib/gcc/nios2-elf/4.1.2/mno-hw-mul/libgcc.a(lib2-mul.o)
 .comment       0x00000000       0x24 ../snake_software_bsp//libhal_bsp.a(alt_load.o)
 .comment       0x00000000       0x24 ../snake_software_bsp//libhal_bsp.a(alt_main.o)
 .comment       0x00000000       0x24 ../snake_software_bsp//libhal_bsp.a(alt_usleep.o)
 .comment       0x00000000       0x24 ../snake_software_bsp//libhal_bsp.a(alt_sys_init.o)
 .comment       0x00000000       0x24 ../snake_software_bsp//libhal_bsp.a(altera_avalon_jtag_uart_fd.o)
 .comment       0x00000000       0x24 ../snake_software_bsp//libhal_bsp.a(altera_avalon_jtag_uart_init.o)
 .comment       0x00000000       0x24 ../snake_software_bsp//libhal_bsp.a(altera_avalon_jtag_uart_ioctl.o)
 .comment       0x00000000       0x24 ../snake_software_bsp//libhal_bsp.a(altera_avalon_jtag_uart_read.o)
 .comment       0x00000000       0x24 ../snake_software_bsp//libhal_bsp.a(altera_avalon_jtag_uart_write.o)
 .comment       0x00000000       0x24 ../snake_software_bsp//libhal_bsp.a(alt_alarm_start.o)
 .comment       0x00000000       0x24 ../snake_software_bsp//libhal_bsp.a(alt_busy_sleep.o)
 .comment       0x00000000       0x24 ../snake_software_bsp//libhal_bsp.a(alt_close.o)
 .comment       0x00000000       0x24 ../snake_software_bsp//libhal_bsp.a(alt_dcache_flush_all.o)
 .comment       0x00000000       0x24 ../snake_software_bsp//libhal_bsp.a(alt_dev.o)
 .comment       0x00000000       0x24 ../snake_software_bsp//libhal_bsp.a(alt_dev_llist_insert.o)
 .comment       0x00000000       0x24 ../snake_software_bsp//libhal_bsp.a(alt_do_ctors.o)
 .comment       0x00000000       0x24 ../snake_software_bsp//libhal_bsp.a(alt_do_dtors.o)
 .comment       0x00000000       0x24 ../snake_software_bsp//libhal_bsp.a(alt_errno.o)
 .comment       0x00000000       0x24 ../snake_software_bsp//libhal_bsp.a(alt_icache_flush_all.o)
 .comment       0x00000000       0x24 ../snake_software_bsp//libhal_bsp.a(alt_iic.o)
 .comment       0x00000000       0x24 ../snake_software_bsp//libhal_bsp.a(alt_iic_isr_register.o)
 .comment       0x00000000       0x24 ../snake_software_bsp//libhal_bsp.a(alt_io_redirect.o)
 .comment       0x00000000       0x24 ../snake_software_bsp//libhal_bsp.a(alt_irq_handler.o)
 .comment       0x00000000       0x24 ../snake_software_bsp//libhal_bsp.a(alt_irq_vars.o)
 .comment       0x00000000       0x24 ../snake_software_bsp//libhal_bsp.a(alt_open.o)
 .comment       0x00000000       0x24 ../snake_software_bsp//libhal_bsp.a(alt_release_fd.o)
 .comment       0x00000000       0x24 ../snake_software_bsp//libhal_bsp.a(alt_tick.o)
 .comment       0x00000000       0x24 ../snake_software_bsp//libhal_bsp.a(altera_nios2_irq.o)
 .comment       0x00000000       0x24 ../snake_software_bsp//libhal_bsp.a(alt_find_dev.o)
 .comment       0x00000000       0x24 ../snake_software_bsp//libhal_bsp.a(alt_find_file.o)
 .comment       0x00000000       0x24 ../snake_software_bsp//libhal_bsp.a(alt_get_fd.o)
 .comment       0x00000000       0x24 /opt/altera/altera12.1/nios2eds/bin/gnu/H-i686-pc-linux-gnu/bin/../lib/gcc/nios2-elf/4.1.2/../../../../nios2-elf/lib/mno-hw-mul/libc.a(lib_a-atexit.o)
 .comment       0x00000000       0x24 /opt/altera/altera12.1/nios2eds/bin/gnu/H-i686-pc-linux-gnu/bin/../lib/gcc/nios2-elf/4.1.2/../../../../nios2-elf/lib/mno-hw-mul/libc.a(lib_a-exit.o)
 .comment       0x00000000       0x24 /opt/altera/altera12.1/nios2eds/bin/gnu/H-i686-pc-linux-gnu/bin/../lib/gcc/nios2-elf/4.1.2/../../../../nios2-elf/lib/mno-hw-mul/libc.a(lib_a-impure.o)
 .comment       0x00000000       0x24 /opt/altera/altera12.1/nios2eds/bin/gnu/H-i686-pc-linux-gnu/bin/../lib/gcc/nios2-elf/4.1.2/../../../../nios2-elf/lib/mno-hw-mul/libc.a(lib_a-int_errno.o)
 .comment       0x00000000       0x24 /opt/altera/altera12.1/nios2eds/bin/gnu/H-i686-pc-linux-gnu/bin/../lib/gcc/nios2-elf/4.1.2/../../../../nios2-elf/lib/mno-hw-mul/libc.a(lib_a-memcmp.o)
 .comment       0x00000000       0x24 /opt/altera/altera12.1/nios2eds/bin/gnu/H-i686-pc-linux-gnu/bin/../lib/gcc/nios2-elf/4.1.2/../../../../nios2-elf/lib/mno-hw-mul/libc.a(lib_a-memcpy.o)
 .comment       0x00000000       0x24 /opt/altera/altera12.1/nios2eds/bin/gnu/H-i686-pc-linux-gnu/bin/../lib/gcc/nios2-elf/4.1.2/../../../../nios2-elf/lib/mno-hw-mul/libc.a(lib_a-strlen.o)
 .comment       0x00000000       0x24 /opt/altera/altera12.1/nios2eds/bin/gnu/H-i686-pc-linux-gnu/bin/../lib/gcc/nios2-elf/4.1.2/../../../../nios2-elf/lib/mno-hw-mul/libc.a(lib_a-__atexit.o)
 .comment       0x00000000       0x24 /opt/altera/altera12.1/nios2eds/bin/gnu/H-i686-pc-linux-gnu/bin/../lib/gcc/nios2-elf/4.1.2/../../../../nios2-elf/lib/mno-hw-mul/libc.a(lib_a-__call_atexit.o)
 .comment       0x00000000       0x24 ../snake_software_bsp//libhal_bsp.a(alt_exit.o)

.debug
 *(.debug)

.line
 *(.line)

.debug_srcinfo
 *(.debug_srcinfo)

.debug_sfnames
 *(.debug_sfnames)

.debug_aranges  0x00000000      0x598
 *(.debug_aranges)
 .debug_aranges
                0x00000000       0x28 ../snake_software_bsp//obj/HAL/src/crt0.o
 .debug_aranges
                0x00000028       0x20 obj/default/main.o
 .debug_aranges
                0x00000048       0x20 /opt/altera/altera12.1/nios2eds/bin/gnu/H-i686-pc-linux-gnu/bin/../lib/gcc/nios2-elf/4.1.2/mno-hw-mul/libgcc.a(lib2-divmod.o)
 .debug_aranges
                0x00000068       0x20 /opt/altera/altera12.1/nios2eds/bin/gnu/H-i686-pc-linux-gnu/bin/../lib/gcc/nios2-elf/4.1.2/mno-hw-mul/libgcc.a(lib2-mul.o)
 .debug_aranges
                0x00000088       0x20 ../snake_software_bsp//libhal_bsp.a(alt_load.o)
 .debug_aranges
                0x000000a8       0x20 ../snake_software_bsp//libhal_bsp.a(alt_main.o)
 .debug_aranges
                0x000000c8       0x20 ../snake_software_bsp//libhal_bsp.a(alt_usleep.o)
 .debug_aranges
                0x000000e8       0x20 ../snake_software_bsp//libhal_bsp.a(alt_sys_init.o)
 .debug_aranges
                0x00000108       0x20 ../snake_software_bsp//libhal_bsp.a(altera_avalon_jtag_uart_fd.o)
 .debug_aranges
                0x00000128       0x20 ../snake_software_bsp//libhal_bsp.a(altera_avalon_jtag_uart_init.o)
 .debug_aranges
                0x00000148       0x20 ../snake_software_bsp//libhal_bsp.a(altera_avalon_jtag_uart_ioctl.o)
 .debug_aranges
                0x00000168       0x20 ../snake_software_bsp//libhal_bsp.a(altera_avalon_jtag_uart_read.o)
 .debug_aranges
                0x00000188       0x20 ../snake_software_bsp//libhal_bsp.a(altera_avalon_jtag_uart_write.o)
 .debug_aranges
                0x000001a8       0x20 ../snake_software_bsp//libhal_bsp.a(alt_alarm_start.o)
 .debug_aranges
                0x000001c8       0x20 ../snake_software_bsp//libhal_bsp.a(alt_busy_sleep.o)
 .debug_aranges
                0x000001e8       0x20 ../snake_software_bsp//libhal_bsp.a(alt_close.o)
 .debug_aranges
                0x00000208       0x20 ../snake_software_bsp//libhal_bsp.a(alt_dcache_flush_all.o)
 .debug_aranges
                0x00000228       0x20 ../snake_software_bsp//libhal_bsp.a(alt_dev.o)
 .debug_aranges
                0x00000248       0x20 ../snake_software_bsp//libhal_bsp.a(alt_dev_llist_insert.o)
 .debug_aranges
                0x00000268       0x20 ../snake_software_bsp//libhal_bsp.a(alt_do_ctors.o)
 .debug_aranges
                0x00000288       0x20 ../snake_software_bsp//libhal_bsp.a(alt_do_dtors.o)
 .debug_aranges
                0x000002a8       0x20 ../snake_software_bsp//libhal_bsp.a(alt_icache_flush_all.o)
 .debug_aranges
                0x000002c8       0x20 ../snake_software_bsp//libhal_bsp.a(alt_iic.o)
 .debug_aranges
                0x000002e8       0x20 ../snake_software_bsp//libhal_bsp.a(alt_iic_isr_register.o)
 .debug_aranges
                0x00000308       0x20 ../snake_software_bsp//libhal_bsp.a(alt_io_redirect.o)
 .debug_aranges
                0x00000328       0x30 ../snake_software_bsp//libhal_bsp.a(alt_irq_entry.o)
 .debug_aranges
                0x00000358       0x28 ../snake_software_bsp//libhal_bsp.a(alt_irq_handler.o)
 .debug_aranges
                0x00000380       0x20 ../snake_software_bsp//libhal_bsp.a(alt_open.o)
 .debug_aranges
                0x000003a0       0x20 ../snake_software_bsp//libhal_bsp.a(alt_release_fd.o)
 .debug_aranges
                0x000003c0       0x20 ../snake_software_bsp//libhal_bsp.a(alt_tick.o)
 .debug_aranges
                0x000003e0       0x20 ../snake_software_bsp//libhal_bsp.a(altera_nios2_irq.o)
 .debug_aranges
                0x00000400       0x38 ../snake_software_bsp//libhal_bsp.a(alt_exception_entry.o)
 .debug_aranges
                0x00000438       0x20 ../snake_software_bsp//libhal_bsp.a(alt_find_dev.o)
 .debug_aranges
                0x00000458       0x20 ../snake_software_bsp//libhal_bsp.a(alt_find_file.o)
 .debug_aranges
                0x00000478       0x20 ../snake_software_bsp//libhal_bsp.a(alt_get_fd.o)
 .debug_aranges
                0x00000498       0x20 /opt/altera/altera12.1/nios2eds/bin/gnu/H-i686-pc-linux-gnu/bin/../lib/gcc/nios2-elf/4.1.2/../../../../nios2-elf/lib/mno-hw-mul/libc.a(lib_a-atexit.o)
 .debug_aranges
                0x000004b8       0x20 /opt/altera/altera12.1/nios2eds/bin/gnu/H-i686-pc-linux-gnu/bin/../lib/gcc/nios2-elf/4.1.2/../../../../nios2-elf/lib/mno-hw-mul/libc.a(lib_a-exit.o)
 .debug_aranges
                0x000004d8       0x20 /opt/altera/altera12.1/nios2eds/bin/gnu/H-i686-pc-linux-gnu/bin/../lib/gcc/nios2-elf/4.1.2/../../../../nios2-elf/lib/mno-hw-mul/libc.a(lib_a-memcmp.o)
 .debug_aranges
                0x000004f8       0x20 /opt/altera/altera12.1/nios2eds/bin/gnu/H-i686-pc-linux-gnu/bin/../lib/gcc/nios2-elf/4.1.2/../../../../nios2-elf/lib/mno-hw-mul/libc.a(lib_a-memcpy.o)
 .debug_aranges
                0x00000518       0x20 /opt/altera/altera12.1/nios2eds/bin/gnu/H-i686-pc-linux-gnu/bin/../lib/gcc/nios2-elf/4.1.2/../../../../nios2-elf/lib/mno-hw-mul/libc.a(lib_a-strlen.o)
 .debug_aranges
                0x00000538       0x20 /opt/altera/altera12.1/nios2eds/bin/gnu/H-i686-pc-linux-gnu/bin/../lib/gcc/nios2-elf/4.1.2/../../../../nios2-elf/lib/mno-hw-mul/libc.a(lib_a-__atexit.o)
 .debug_aranges
                0x00000558       0x20 /opt/altera/altera12.1/nios2eds/bin/gnu/H-i686-pc-linux-gnu/bin/../lib/gcc/nios2-elf/4.1.2/../../../../nios2-elf/lib/mno-hw-mul/libc.a(lib_a-__call_atexit.o)
 .debug_aranges
                0x00000578       0x20 ../snake_software_bsp//libhal_bsp.a(alt_exit.o)

.debug_pubnames
                0x00000000     0x1425
 *(.debug_pubnames)
 .debug_pubnames
                0x00000000      0xc02 obj/default/main.o
 .debug_pubnames
                0x00000c02       0x48 /opt/altera/altera12.1/nios2eds/bin/gnu/H-i686-pc-linux-gnu/bin/../lib/gcc/nios2-elf/4.1.2/mno-hw-mul/libgcc.a(lib2-divmod.o)
 .debug_pubnames
                0x00000c4a       0x1f /opt/altera/altera12.1/nios2eds/bin/gnu/H-i686-pc-linux-gnu/bin/../lib/gcc/nios2-elf/4.1.2/mno-hw-mul/libgcc.a(lib2-mul.o)
 .debug_pubnames
                0x00000c69       0x1f ../snake_software_bsp//libhal_bsp.a(alt_load.o)
 .debug_pubnames
                0x00000c88       0x46 ../snake_software_bsp//libhal_bsp.a(alt_main.o)
 .debug_pubnames
                0x00000cce       0x1d ../snake_software_bsp//libhal_bsp.a(alt_usleep.o)
 .debug_pubnames
                0x00000ceb       0x34 ../snake_software_bsp//libhal_bsp.a(alt_sys_init.o)
 .debug_pubnames
                0x00000d1f       0xa5 ../snake_software_bsp//libhal_bsp.a(altera_avalon_jtag_uart_fd.o)
 .debug_pubnames
                0x00000dc4       0x55 ../snake_software_bsp//libhal_bsp.a(altera_avalon_jtag_uart_init.o)
 .debug_pubnames
                0x00000e19       0x34 ../snake_software_bsp//libhal_bsp.a(altera_avalon_jtag_uart_ioctl.o)
 .debug_pubnames
                0x00000e4d       0x33 ../snake_software_bsp//libhal_bsp.a(altera_avalon_jtag_uart_read.o)
 .debug_pubnames
                0x00000e80       0x34 ../snake_software_bsp//libhal_bsp.a(altera_avalon_jtag_uart_write.o)
 .debug_pubnames
                0x00000eb4       0x26 ../snake_software_bsp//libhal_bsp.a(alt_alarm_start.o)
 .debug_pubnames
                0x00000eda       0x25 ../snake_software_bsp//libhal_bsp.a(alt_busy_sleep.o)
 .debug_pubnames
                0x00000eff       0x1c ../snake_software_bsp//libhal_bsp.a(alt_close.o)
 .debug_pubnames
                0x00000f1b       0x2b ../snake_software_bsp//libhal_bsp.a(alt_dcache_flush_all.o)
 .debug_pubnames
                0x00000f46       0x63 ../snake_software_bsp//libhal_bsp.a(alt_dev.o)
 .debug_pubnames
                0x00000fa9       0x2b ../snake_software_bsp//libhal_bsp.a(alt_dev_llist_insert.o)
 .debug_pubnames
                0x00000fd4       0x20 ../snake_software_bsp//libhal_bsp.a(alt_do_ctors.o)
 .debug_pubnames
                0x00000ff4       0x20 ../snake_software_bsp//libhal_bsp.a(alt_do_dtors.o)
 .debug_pubnames
                0x00001014       0x20 ../snake_software_bsp//libhal_bsp.a(alt_errno.o)
 .debug_pubnames
                0x00001034       0x2b ../snake_software_bsp//libhal_bsp.a(alt_icache_flush_all.o)
 .debug_pubnames
                0x0000105f       0x6e ../snake_software_bsp//libhal_bsp.a(alt_iic.o)
 .debug_pubnames
                0x000010cd       0x2b ../snake_software_bsp//libhal_bsp.a(alt_iic_isr_register.o)
 .debug_pubnames
                0x000010f8       0x26 ../snake_software_bsp//libhal_bsp.a(alt_io_redirect.o)
 .debug_pubnames
                0x0000111e       0x32 ../snake_software_bsp//libhal_bsp.a(alt_irq_handler.o)
 .debug_pubnames
                0x00001150       0x3b ../snake_software_bsp//libhal_bsp.a(alt_irq_vars.o)
 .debug_pubnames
                0x0000118b       0x1b ../snake_software_bsp//libhal_bsp.a(alt_open.o)
 .debug_pubnames
                0x000011a6       0x25 ../snake_software_bsp//libhal_bsp.a(alt_release_fd.o)
 .debug_pubnames
                0x000011cb       0x68 ../snake_software_bsp//libhal_bsp.a(alt_tick.o)
 .debug_pubnames
                0x00001233       0x2c ../snake_software_bsp//libhal_bsp.a(altera_nios2_irq.o)
 .debug_pubnames
                0x0000125f       0x23 ../snake_software_bsp//libhal_bsp.a(alt_find_dev.o)
 .debug_pubnames
                0x00001282       0x24 ../snake_software_bsp//libhal_bsp.a(alt_find_file.o)
 .debug_pubnames
                0x000012a6       0x21 ../snake_software_bsp//libhal_bsp.a(alt_get_fd.o)
 .debug_pubnames
                0x000012c7       0x2a /opt/altera/altera12.1/nios2eds/bin/gnu/H-i686-pc-linux-gnu/bin/../lib/gcc/nios2-elf/4.1.2/../../../../nios2-elf/lib/mno-hw-mul/libc.a(lib_a-atexit.o)
 .debug_pubnames
                0x000012f1       0x1b /opt/altera/altera12.1/nios2eds/bin/gnu/H-i686-pc-linux-gnu/bin/../lib/gcc/nios2-elf/4.1.2/../../../../nios2-elf/lib/mno-hw-mul/libc.a(lib_a-exit.o)
 .debug_pubnames
                0x0000130c       0x39 /opt/altera/altera12.1/nios2eds/bin/gnu/H-i686-pc-linux-gnu/bin/../lib/gcc/nios2-elf/4.1.2/../../../../nios2-elf/lib/mno-hw-mul/libc.a(lib_a-impure.o)
 .debug_pubnames
                0x00001345       0x1c /opt/altera/altera12.1/nios2eds/bin/gnu/H-i686-pc-linux-gnu/bin/../lib/gcc/nios2-elf/4.1.2/../../../../nios2-elf/lib/mno-hw-mul/libc.a(lib_a-int_errno.o)
 .debug_pubnames
                0x00001361       0x1d /opt/altera/altera12.1/nios2eds/bin/gnu/H-i686-pc-linux-gnu/bin/../lib/gcc/nios2-elf/4.1.2/../../../../nios2-elf/lib/mno-hw-mul/libc.a(lib_a-memcmp.o)
 .debug_pubnames
                0x0000137e       0x1d /opt/altera/altera12.1/nios2eds/bin/gnu/H-i686-pc-linux-gnu/bin/../lib/gcc/nios2-elf/4.1.2/../../../../nios2-elf/lib/mno-hw-mul/libc.a(lib_a-memcpy.o)
 .debug_pubnames
                0x0000139b       0x1d /opt/altera/altera12.1/nios2eds/bin/gnu/H-i686-pc-linux-gnu/bin/../lib/gcc/nios2-elf/4.1.2/../../../../nios2-elf/lib/mno-hw-mul/libc.a(lib_a-strlen.o)
 .debug_pubnames
                0x000013b8       0x2a /opt/altera/altera12.1/nios2eds/bin/gnu/H-i686-pc-linux-gnu/bin/../lib/gcc/nios2-elf/4.1.2/../../../../nios2-elf/lib/mno-hw-mul/libc.a(lib_a-__atexit.o)
 .debug_pubnames
                0x000013e2       0x27 /opt/altera/altera12.1/nios2eds/bin/gnu/H-i686-pc-linux-gnu/bin/../lib/gcc/nios2-elf/4.1.2/../../../../nios2-elf/lib/mno-hw-mul/libc.a(lib_a-__call_atexit.o)
 .debug_pubnames
                0x00001409       0x1c ../snake_software_bsp//libhal_bsp.a(alt_exit.o)

.debug_info     0x00000000     0xcd08
 *(.debug_info .gnu.linkonce.wi.*)
 .debug_info    0x00000000       0x7d ../snake_software_bsp//obj/HAL/src/crt0.o
 .debug_info    0x0000007d      0x123 obj/default/hello_world.o
 .debug_info    0x000001a0     0x2a0a obj/default/main.o
 .debug_info    0x00002baa      0x21c /opt/altera/altera12.1/nios2eds/bin/gnu/H-i686-pc-linux-gnu/bin/../lib/gcc/nios2-elf/4.1.2/mno-hw-mul/libgcc.a(lib2-divmod.o)
 .debug_info    0x00002dc6       0xf3 /opt/altera/altera12.1/nios2eds/bin/gnu/H-i686-pc-linux-gnu/bin/../lib/gcc/nios2-elf/4.1.2/mno-hw-mul/libgcc.a(lib2-mul.o)
 .debug_info    0x00002eb9      0x28f ../snake_software_bsp//libhal_bsp.a(alt_load.o)
 .debug_info    0x00003148      0x227 ../snake_software_bsp//libhal_bsp.a(alt_main.o)
 .debug_info    0x0000336f      0x16a ../snake_software_bsp//libhal_bsp.a(alt_usleep.o)
 .debug_info    0x000034d9      0x6da ../snake_software_bsp//libhal_bsp.a(alt_sys_init.o)
 .debug_info    0x00003bb3      0x7db ../snake_software_bsp//libhal_bsp.a(altera_avalon_jtag_uart_fd.o)
 .debug_info    0x0000438e      0x603 ../snake_software_bsp//libhal_bsp.a(altera_avalon_jtag_uart_init.o)
 .debug_info    0x00004991      0x445 ../snake_software_bsp//libhal_bsp.a(altera_avalon_jtag_uart_ioctl.o)
 .debug_info    0x00004dd6      0x548 ../snake_software_bsp//libhal_bsp.a(altera_avalon_jtag_uart_read.o)
 .debug_info    0x0000531e      0x540 ../snake_software_bsp//libhal_bsp.a(altera_avalon_jtag_uart_write.o)
 .debug_info    0x0000585e      0x444 ../snake_software_bsp//libhal_bsp.a(alt_alarm_start.o)
 .debug_info    0x00005ca2      0x1ad ../snake_software_bsp//libhal_bsp.a(alt_busy_sleep.o)
 .debug_info    0x00005e4f      0x469 ../snake_software_bsp//libhal_bsp.a(alt_close.o)
 .debug_info    0x000062b8      0x15e ../snake_software_bsp//libhal_bsp.a(alt_dcache_flush_all.o)
 .debug_info    0x00006416      0x681 ../snake_software_bsp//libhal_bsp.a(alt_dev.o)
 .debug_info    0x00006a97      0x2b9 ../snake_software_bsp//libhal_bsp.a(alt_dev_llist_insert.o)
 .debug_info    0x00006d50      0x111 ../snake_software_bsp//libhal_bsp.a(alt_do_ctors.o)
 .debug_info    0x00006e61      0x110 ../snake_software_bsp//libhal_bsp.a(alt_do_dtors.o)
 .debug_info    0x00006f71      0x166 ../snake_software_bsp//libhal_bsp.a(alt_errno.o)
 .debug_info    0x000070d7      0x15e ../snake_software_bsp//libhal_bsp.a(alt_icache_flush_all.o)
 .debug_info    0x00007235      0x495 ../snake_software_bsp//libhal_bsp.a(alt_iic.o)
 .debug_info    0x000076ca      0x316 ../snake_software_bsp//libhal_bsp.a(alt_iic_isr_register.o)
 .debug_info    0x000079e0      0x697 ../snake_software_bsp//libhal_bsp.a(alt_io_redirect.o)
 .debug_info    0x00008077       0x86 ../snake_software_bsp//libhal_bsp.a(alt_irq_entry.o)
 .debug_info    0x000080fd      0x277 ../snake_software_bsp//libhal_bsp.a(alt_irq_handler.o)
 .debug_info    0x00008374      0x169 ../snake_software_bsp//libhal_bsp.a(alt_irq_vars.o)
 .debug_info    0x000084dd      0x527 ../snake_software_bsp//libhal_bsp.a(alt_open.o)
 .debug_info    0x00008a04      0x3f4 ../snake_software_bsp//libhal_bsp.a(alt_release_fd.o)
 .debug_info    0x00008df8      0x400 ../snake_software_bsp//libhal_bsp.a(alt_tick.o)
 .debug_info    0x000091f8      0x15b ../snake_software_bsp//libhal_bsp.a(altera_nios2_irq.o)
 .debug_info    0x00009353       0x8c ../snake_software_bsp//libhal_bsp.a(alt_exception_entry.o)
 .debug_info    0x000093df      0x41a ../snake_software_bsp//libhal_bsp.a(alt_find_dev.o)
 .debug_info    0x000097f9      0x421 ../snake_software_bsp//libhal_bsp.a(alt_find_file.o)
 .debug_info    0x00009c1a      0x462 ../snake_software_bsp//libhal_bsp.a(alt_get_fd.o)
 .debug_info    0x0000a07c      0x181 /opt/altera/altera12.1/nios2eds/bin/gnu/H-i686-pc-linux-gnu/bin/../lib/gcc/nios2-elf/4.1.2/../../../../nios2-elf/lib/mno-hw-mul/libc.a(lib_a-atexit.o)
 .debug_info    0x0000a1fd      0x93f /opt/altera/altera12.1/nios2eds/bin/gnu/H-i686-pc-linux-gnu/bin/../lib/gcc/nios2-elf/4.1.2/../../../../nios2-elf/lib/mno-hw-mul/libc.a(lib_a-exit.o)
 .debug_info    0x0000ab3c      0x93d /opt/altera/altera12.1/nios2eds/bin/gnu/H-i686-pc-linux-gnu/bin/../lib/gcc/nios2-elf/4.1.2/../../../../nios2-elf/lib/mno-hw-mul/libc.a(lib_a-impure.o)
 .debug_info    0x0000b479       0x8c /opt/altera/altera12.1/nios2eds/bin/gnu/H-i686-pc-linux-gnu/bin/../lib/gcc/nios2-elf/4.1.2/../../../../nios2-elf/lib/mno-hw-mul/libc.a(lib_a-int_errno.o)
 .debug_info    0x0000b505      0x115 /opt/altera/altera12.1/nios2eds/bin/gnu/H-i686-pc-linux-gnu/bin/../lib/gcc/nios2-elf/4.1.2/../../../../nios2-elf/lib/mno-hw-mul/libc.a(lib_a-memcmp.o)
 .debug_info    0x0000b61a      0x106 /opt/altera/altera12.1/nios2eds/bin/gnu/H-i686-pc-linux-gnu/bin/../lib/gcc/nios2-elf/4.1.2/../../../../nios2-elf/lib/mno-hw-mul/libc.a(lib_a-memcpy.o)
 .debug_info    0x0000b720       0xdb /opt/altera/altera12.1/nios2eds/bin/gnu/H-i686-pc-linux-gnu/bin/../lib/gcc/nios2-elf/4.1.2/../../../../nios2-elf/lib/mno-hw-mul/libc.a(lib_a-strlen.o)
 .debug_info    0x0000b7fb      0x99c /opt/altera/altera12.1/nios2eds/bin/gnu/H-i686-pc-linux-gnu/bin/../lib/gcc/nios2-elf/4.1.2/../../../../nios2-elf/lib/mno-hw-mul/libc.a(lib_a-__atexit.o)
 .debug_info    0x0000c197      0x9e2 /opt/altera/altera12.1/nios2eds/bin/gnu/H-i686-pc-linux-gnu/bin/../lib/gcc/nios2-elf/4.1.2/../../../../nios2-elf/lib/mno-hw-mul/libc.a(lib_a-__call_atexit.o)
 .debug_info    0x0000cb79      0x18f ../snake_software_bsp//libhal_bsp.a(alt_exit.o)

.debug_abbrev   0x00000000     0x279d
 *(.debug_abbrev)
 .debug_abbrev  0x00000000       0x12 ../snake_software_bsp//obj/HAL/src/crt0.o
 .debug_abbrev  0x00000012       0x2a obj/default/hello_world.o
 .debug_abbrev  0x0000003c      0x1f7 obj/default/main.o
 .debug_abbrev  0x00000233       0xe0 /opt/altera/altera12.1/nios2eds/bin/gnu/H-i686-pc-linux-gnu/bin/../lib/gcc/nios2-elf/4.1.2/mno-hw-mul/libgcc.a(lib2-divmod.o)
 .debug_abbrev  0x00000313       0x7b /opt/altera/altera12.1/nios2eds/bin/gnu/H-i686-pc-linux-gnu/bin/../lib/gcc/nios2-elf/4.1.2/mno-hw-mul/libgcc.a(lib2-mul.o)
 .debug_abbrev  0x0000038e       0x88 ../snake_software_bsp//libhal_bsp.a(alt_load.o)
 .debug_abbrev  0x00000416       0xb7 ../snake_software_bsp//libhal_bsp.a(alt_main.o)
 .debug_abbrev  0x000004cd       0x5d ../snake_software_bsp//libhal_bsp.a(alt_usleep.o)
 .debug_abbrev  0x0000052a      0x142 ../snake_software_bsp//libhal_bsp.a(alt_sys_init.o)
 .debug_abbrev  0x0000066c       0xf7 ../snake_software_bsp//libhal_bsp.a(altera_avalon_jtag_uart_fd.o)
 .debug_abbrev  0x00000763      0x17c ../snake_software_bsp//libhal_bsp.a(altera_avalon_jtag_uart_init.o)
 .debug_abbrev  0x000008df       0xf0 ../snake_software_bsp//libhal_bsp.a(altera_avalon_jtag_uart_ioctl.o)
 .debug_abbrev  0x000009cf      0x191 ../snake_software_bsp//libhal_bsp.a(altera_avalon_jtag_uart_read.o)
 .debug_abbrev  0x00000b60      0x18d ../snake_software_bsp//libhal_bsp.a(altera_avalon_jtag_uart_write.o)
 .debug_abbrev  0x00000ced      0x172 ../snake_software_bsp//libhal_bsp.a(alt_alarm_start.o)
 .debug_abbrev  0x00000e5f       0x6c ../snake_software_bsp//libhal_bsp.a(alt_busy_sleep.o)
 .debug_abbrev  0x00000ecb       0xfb ../snake_software_bsp//libhal_bsp.a(alt_close.o)
 .debug_abbrev  0x00000fc6       0x3f ../snake_software_bsp//libhal_bsp.a(alt_dcache_flush_all.o)
 .debug_abbrev  0x00001005       0xc7 ../snake_software_bsp//libhal_bsp.a(alt_dev.o)
 .debug_abbrev  0x000010cc       0xf6 ../snake_software_bsp//libhal_bsp.a(alt_dev_llist_insert.o)
 .debug_abbrev  0x000011c2       0x76 ../snake_software_bsp//libhal_bsp.a(alt_do_ctors.o)
 .debug_abbrev  0x00001238       0x76 ../snake_software_bsp//libhal_bsp.a(alt_do_dtors.o)
 .debug_abbrev  0x000012ae       0x5e ../snake_software_bsp//libhal_bsp.a(alt_errno.o)
 .debug_abbrev  0x0000130c       0x3f ../snake_software_bsp//libhal_bsp.a(alt_icache_flush_all.o)
 .debug_abbrev  0x0000134b      0x134 ../snake_software_bsp//libhal_bsp.a(alt_iic.o)
 .debug_abbrev  0x0000147f      0x14e ../snake_software_bsp//libhal_bsp.a(alt_iic_isr_register.o)
 .debug_abbrev  0x000015cd       0xf0 ../snake_software_bsp//libhal_bsp.a(alt_io_redirect.o)
 .debug_abbrev  0x000016bd       0x12 ../snake_software_bsp//libhal_bsp.a(alt_irq_entry.o)
 .debug_abbrev  0x000016cf      0x10c ../snake_software_bsp//libhal_bsp.a(alt_irq_handler.o)
 .debug_abbrev  0x000017db       0x44 ../snake_software_bsp//libhal_bsp.a(alt_irq_vars.o)
 .debug_abbrev  0x0000181f      0x112 ../snake_software_bsp//libhal_bsp.a(alt_open.o)
 .debug_abbrev  0x00001931       0xc1 ../snake_software_bsp//libhal_bsp.a(alt_release_fd.o)
 .debug_abbrev  0x000019f2      0x150 ../snake_software_bsp//libhal_bsp.a(alt_tick.o)
 .debug_abbrev  0x00001b42       0x3f ../snake_software_bsp//libhal_bsp.a(altera_nios2_irq.o)
 .debug_abbrev  0x00001b81       0x12 ../snake_software_bsp//libhal_bsp.a(alt_exception_entry.o)
 .debug_abbrev  0x00001b93       0xcf ../snake_software_bsp//libhal_bsp.a(alt_find_dev.o)
 .debug_abbrev  0x00001c62       0xcf ../snake_software_bsp//libhal_bsp.a(alt_find_file.o)
 .debug_abbrev  0x00001d31       0xfb ../snake_software_bsp//libhal_bsp.a(alt_get_fd.o)
 .debug_abbrev  0x00001e2c       0xb7 /opt/altera/altera12.1/nios2eds/bin/gnu/H-i686-pc-linux-gnu/bin/../lib/gcc/nios2-elf/4.1.2/../../../../nios2-elf/lib/mno-hw-mul/libc.a(lib_a-atexit.o)
 .debug_abbrev  0x00001ee3      0x16e /opt/altera/altera12.1/nios2eds/bin/gnu/H-i686-pc-linux-gnu/bin/../lib/gcc/nios2-elf/4.1.2/../../../../nios2-elf/lib/mno-hw-mul/libc.a(lib_a-exit.o)
 .debug_abbrev  0x00002051      0x157 /opt/altera/altera12.1/nios2eds/bin/gnu/H-i686-pc-linux-gnu/bin/../lib/gcc/nios2-elf/4.1.2/../../../../nios2-elf/lib/mno-hw-mul/libc.a(lib_a-impure.o)
 .debug_abbrev  0x000021a8       0x3b /opt/altera/altera12.1/nios2eds/bin/gnu/H-i686-pc-linux-gnu/bin/../lib/gcc/nios2-elf/4.1.2/../../../../nios2-elf/lib/mno-hw-mul/libc.a(lib_a-int_errno.o)
 .debug_abbrev  0x000021e3       0x7c /opt/altera/altera12.1/nios2eds/bin/gnu/H-i686-pc-linux-gnu/bin/../lib/gcc/nios2-elf/4.1.2/../../../../nios2-elf/lib/mno-hw-mul/libc.a(lib_a-memcmp.o)
 .debug_abbrev  0x0000225f       0xb5 /opt/altera/altera12.1/nios2eds/bin/gnu/H-i686-pc-linux-gnu/bin/../lib/gcc/nios2-elf/4.1.2/../../../../nios2-elf/lib/mno-hw-mul/libc.a(lib_a-memcpy.o)
 .debug_abbrev  0x00002314       0x8b /opt/altera/altera12.1/nios2eds/bin/gnu/H-i686-pc-linux-gnu/bin/../lib/gcc/nios2-elf/4.1.2/../../../../nios2-elf/lib/mno-hw-mul/libc.a(lib_a-strlen.o)
 .debug_abbrev  0x0000239f      0x1ae /opt/altera/altera12.1/nios2eds/bin/gnu/H-i686-pc-linux-gnu/bin/../lib/gcc/nios2-elf/4.1.2/../../../../nios2-elf/lib/mno-hw-mul/libc.a(lib_a-__atexit.o)
 .debug_abbrev  0x0000254d      0x1de /opt/altera/altera12.1/nios2eds/bin/gnu/H-i686-pc-linux-gnu/bin/../lib/gcc/nios2-elf/4.1.2/../../../../nios2-elf/lib/mno-hw-mul/libc.a(lib_a-__call_atexit.o)
 .debug_abbrev  0x0000272b       0x72 ../snake_software_bsp//libhal_bsp.a(alt_exit.o)

.debug_line     0x00000000     0x8e04
 *(.debug_line)
 .debug_line    0x00000000       0x66 ../snake_software_bsp//obj/HAL/src/crt0.o
 .debug_line    0x00000066      0x1ab obj/default/hello_world.o
 .debug_line    0x00000211     0x2472 obj/default/main.o
 .debug_line    0x00002683      0x2c3 /opt/altera/altera12.1/nios2eds/bin/gnu/H-i686-pc-linux-gnu/bin/../lib/gcc/nios2-elf/4.1.2/mno-hw-mul/libgcc.a(lib2-divmod.o)
 .debug_line    0x00002946      0x18e /opt/altera/altera12.1/nios2eds/bin/gnu/H-i686-pc-linux-gnu/bin/../lib/gcc/nios2-elf/4.1.2/mno-hw-mul/libgcc.a(lib2-mul.o)
 .debug_line    0x00002ad4      0x22b ../snake_software_bsp//libhal_bsp.a(alt_load.o)
 .debug_line    0x00002cff      0x2de ../snake_software_bsp//libhal_bsp.a(alt_main.o)
 .debug_line    0x00002fdd      0x220 ../snake_software_bsp//libhal_bsp.a(alt_usleep.o)
 .debug_line    0x000031fd      0x2ba ../snake_software_bsp//libhal_bsp.a(alt_sys_init.o)
 .debug_line    0x000034b7      0x221 ../snake_software_bsp//libhal_bsp.a(altera_avalon_jtag_uart_fd.o)
 .debug_line    0x000036d8      0x4bf ../snake_software_bsp//libhal_bsp.a(altera_avalon_jtag_uart_init.o)
 .debug_line    0x00003b97      0x32b ../snake_software_bsp//libhal_bsp.a(altera_avalon_jtag_uart_ioctl.o)
 .debug_line    0x00003ec2      0x40b ../snake_software_bsp//libhal_bsp.a(altera_avalon_jtag_uart_read.o)
 .debug_line    0x000042cd      0x419 ../snake_software_bsp//libhal_bsp.a(altera_avalon_jtag_uart_write.o)
 .debug_line    0x000046e6      0x2f0 ../snake_software_bsp//libhal_bsp.a(alt_alarm_start.o)
 .debug_line    0x000049d6      0x27a ../snake_software_bsp//libhal_bsp.a(alt_busy_sleep.o)
 .debug_line    0x00004c50      0x2ad ../snake_software_bsp//libhal_bsp.a(alt_close.o)
 .debug_line    0x00004efd      0x1c9 ../snake_software_bsp//libhal_bsp.a(alt_dcache_flush_all.o)
 .debug_line    0x000050c6      0x268 ../snake_software_bsp//libhal_bsp.a(alt_dev.o)
 .debug_line    0x0000532e      0x26e ../snake_software_bsp//libhal_bsp.a(alt_dev_llist_insert.o)
 .debug_line    0x0000559c       0x83 ../snake_software_bsp//libhal_bsp.a(alt_do_ctors.o)
 .debug_line    0x0000561f       0x83 ../snake_software_bsp//libhal_bsp.a(alt_do_dtors.o)
 .debug_line    0x000056a2      0x1be ../snake_software_bsp//libhal_bsp.a(alt_errno.o)
 .debug_line    0x00005860      0x1c9 ../snake_software_bsp//libhal_bsp.a(alt_icache_flush_all.o)
 .debug_line    0x00005a29      0x2dc ../snake_software_bsp//libhal_bsp.a(alt_iic.o)
 .debug_line    0x00005d05      0x25d ../snake_software_bsp//libhal_bsp.a(alt_iic_isr_register.o)
 .debug_line    0x00005f62      0x2c8 ../snake_software_bsp//libhal_bsp.a(alt_io_redirect.o)
 .debug_line    0x0000622a       0x6b ../snake_software_bsp//libhal_bsp.a(alt_irq_entry.o)
 .debug_line    0x00006295      0x25c ../snake_software_bsp//libhal_bsp.a(alt_irq_handler.o)
 .debug_line    0x000064f1       0x72 ../snake_software_bsp//libhal_bsp.a(alt_irq_vars.o)
 .debug_line    0x00006563      0x313 ../snake_software_bsp//libhal_bsp.a(alt_open.o)
 .debug_line    0x00006876       0xed ../snake_software_bsp//libhal_bsp.a(alt_release_fd.o)
 .debug_line    0x00006963      0x2f0 ../snake_software_bsp//libhal_bsp.a(alt_tick.o)
 .debug_line    0x00006c53      0x1dd ../snake_software_bsp//libhal_bsp.a(altera_nios2_irq.o)
 .debug_line    0x00006e30       0xab ../snake_software_bsp//libhal_bsp.a(alt_exception_entry.o)
 .debug_line    0x00006edb      0x27f ../snake_software_bsp//libhal_bsp.a(alt_find_dev.o)
 .debug_line    0x0000715a      0x290 ../snake_software_bsp//libhal_bsp.a(alt_find_file.o)
 .debug_line    0x000073ea      0x2ab ../snake_software_bsp//libhal_bsp.a(alt_get_fd.o)
 .debug_line    0x00007695      0x1fd /opt/altera/altera12.1/nios2eds/bin/gnu/H-i686-pc-linux-gnu/bin/../lib/gcc/nios2-elf/4.1.2/../../../../nios2-elf/lib/mno-hw-mul/libc.a(lib_a-atexit.o)
 .debug_line    0x00007892      0x235 /opt/altera/altera12.1/nios2eds/bin/gnu/H-i686-pc-linux-gnu/bin/../lib/gcc/nios2-elf/4.1.2/../../../../nios2-elf/lib/mno-hw-mul/libc.a(lib_a-exit.o)
 .debug_line    0x00007ac7      0x227 /opt/altera/altera12.1/nios2eds/bin/gnu/H-i686-pc-linux-gnu/bin/../lib/gcc/nios2-elf/4.1.2/../../../../nios2-elf/lib/mno-hw-mul/libc.a(lib_a-impure.o)
 .debug_line    0x00007cee      0x1dc /opt/altera/altera12.1/nios2eds/bin/gnu/H-i686-pc-linux-gnu/bin/../lib/gcc/nios2-elf/4.1.2/../../../../nios2-elf/lib/mno-hw-mul/libc.a(lib_a-int_errno.o)
 .debug_line    0x00007eca      0x299 /opt/altera/altera12.1/nios2eds/bin/gnu/H-i686-pc-linux-gnu/bin/../lib/gcc/nios2-elf/4.1.2/../../../../nios2-elf/lib/mno-hw-mul/libc.a(lib_a-memcmp.o)
 .debug_line    0x00008163      0x1ac /opt/altera/altera12.1/nios2eds/bin/gnu/H-i686-pc-linux-gnu/bin/../lib/gcc/nios2-elf/4.1.2/../../../../nios2-elf/lib/mno-hw-mul/libc.a(lib_a-memcpy.o)
 .debug_line    0x0000830f      0x267 /opt/altera/altera12.1/nios2eds/bin/gnu/H-i686-pc-linux-gnu/bin/../lib/gcc/nios2-elf/4.1.2/../../../../nios2-elf/lib/mno-hw-mul/libc.a(lib_a-strlen.o)
 .debug_line    0x00008576      0x310 /opt/altera/altera12.1/nios2eds/bin/gnu/H-i686-pc-linux-gnu/bin/../lib/gcc/nios2-elf/4.1.2/../../../../nios2-elf/lib/mno-hw-mul/libc.a(lib_a-__atexit.o)
 .debug_line    0x00008886      0x364 /opt/altera/altera12.1/nios2eds/bin/gnu/H-i686-pc-linux-gnu/bin/../lib/gcc/nios2-elf/4.1.2/../../../../nios2-elf/lib/mno-hw-mul/libc.a(lib_a-__call_atexit.o)
 .debug_line    0x00008bea      0x21a ../snake_software_bsp//libhal_bsp.a(alt_exit.o)

.debug_frame    0x00000000     0x11fc
 *(.debug_frame)
 .debug_frame   0x00000000      0x8f8 obj/default/main.o
 .debug_frame   0x000008f8       0x70 /opt/altera/altera12.1/nios2eds/bin/gnu/H-i686-pc-linux-gnu/bin/../lib/gcc/nios2-elf/4.1.2/mno-hw-mul/libgcc.a(lib2-divmod.o)
 .debug_frame   0x00000968       0x20 /opt/altera/altera12.1/nios2eds/bin/gnu/H-i686-pc-linux-gnu/bin/../lib/gcc/nios2-elf/4.1.2/mno-hw-mul/libgcc.a(lib2-mul.o)
 .debug_frame   0x00000988       0x48 ../snake_software_bsp//libhal_bsp.a(alt_load.o)
 .debug_frame   0x000009d0       0x2c ../snake_software_bsp//libhal_bsp.a(alt_main.o)
 .debug_frame   0x000009fc       0x2c ../snake_software_bsp//libhal_bsp.a(alt_usleep.o)
 .debug_frame   0x00000a28       0x64 ../snake_software_bsp//libhal_bsp.a(alt_sys_init.o)
 .debug_frame   0x00000a8c       0x80 ../snake_software_bsp//libhal_bsp.a(altera_avalon_jtag_uart_fd.o)
 .debug_frame   0x00000b0c       0x80 ../snake_software_bsp//libhal_bsp.a(altera_avalon_jtag_uart_init.o)
 .debug_frame   0x00000b8c       0x2c ../snake_software_bsp//libhal_bsp.a(altera_avalon_jtag_uart_ioctl.o)
 .debug_frame   0x00000bb8       0x2c ../snake_software_bsp//libhal_bsp.a(altera_avalon_jtag_uart_read.o)
 .debug_frame   0x00000be4       0x2c ../snake_software_bsp//libhal_bsp.a(altera_avalon_jtag_uart_write.o)
 .debug_frame   0x00000c10       0x2c ../snake_software_bsp//libhal_bsp.a(alt_alarm_start.o)
 .debug_frame   0x00000c3c       0x2c ../snake_software_bsp//libhal_bsp.a(alt_busy_sleep.o)
 .debug_frame   0x00000c68       0x48 ../snake_software_bsp//libhal_bsp.a(alt_close.o)
 .debug_frame   0x00000cb0       0x2c ../snake_software_bsp//libhal_bsp.a(alt_dcache_flush_all.o)
 .debug_frame   0x00000cdc       0x2c ../snake_software_bsp//libhal_bsp.a(alt_dev.o)
 .debug_frame   0x00000d08       0x48 ../snake_software_bsp//libhal_bsp.a(alt_dev_llist_insert.o)
 .debug_frame   0x00000d50       0x2c ../snake_software_bsp//libhal_bsp.a(alt_do_ctors.o)
 .debug_frame   0x00000d7c       0x2c ../snake_software_bsp//libhal_bsp.a(alt_do_dtors.o)
 .debug_frame   0x00000da8       0x2c ../snake_software_bsp//libhal_bsp.a(alt_icache_flush_all.o)
 .debug_frame   0x00000dd4       0x80 ../snake_software_bsp//libhal_bsp.a(alt_iic.o)
 .debug_frame   0x00000e54       0x2c ../snake_software_bsp//libhal_bsp.a(alt_iic_isr_register.o)
 .debug_frame   0x00000e80       0x4c ../snake_software_bsp//libhal_bsp.a(alt_io_redirect.o)
 .debug_frame   0x00000ecc       0x2c ../snake_software_bsp//libhal_bsp.a(alt_irq_handler.o)
 .debug_frame   0x00000ef8       0x68 ../snake_software_bsp//libhal_bsp.a(alt_open.o)
 .debug_frame   0x00000f60       0x30 ../snake_software_bsp//libhal_bsp.a(alt_release_fd.o)
 .debug_frame   0x00000f90       0x48 ../snake_software_bsp//libhal_bsp.a(alt_tick.o)
 .debug_frame   0x00000fd8       0x2c ../snake_software_bsp//libhal_bsp.a(altera_nios2_irq.o)
 .debug_frame   0x00001004       0x2c ../snake_software_bsp//libhal_bsp.a(alt_find_dev.o)
 .debug_frame   0x00001030       0x2c ../snake_software_bsp//libhal_bsp.a(alt_find_file.o)
 .debug_frame   0x0000105c       0x30 ../snake_software_bsp//libhal_bsp.a(alt_get_fd.o)
 .debug_frame   0x0000108c       0x20 /opt/altera/altera12.1/nios2eds/bin/gnu/H-i686-pc-linux-gnu/bin/../lib/gcc/nios2-elf/4.1.2/../../../../nios2-elf/lib/mno-hw-mul/libc.a(lib_a-atexit.o)
 .debug_frame   0x000010ac       0x28 /opt/altera/altera12.1/nios2eds/bin/gnu/H-i686-pc-linux-gnu/bin/../lib/gcc/nios2-elf/4.1.2/../../../../nios2-elf/lib/mno-hw-mul/libc.a(lib_a-exit.o)
 .debug_frame   0x000010d4       0x20 /opt/altera/altera12.1/nios2eds/bin/gnu/H-i686-pc-linux-gnu/bin/../lib/gcc/nios2-elf/4.1.2/../../../../nios2-elf/lib/mno-hw-mul/libc.a(lib_a-memcmp.o)
 .debug_frame   0x000010f4       0x20 /opt/altera/altera12.1/nios2eds/bin/gnu/H-i686-pc-linux-gnu/bin/../lib/gcc/nios2-elf/4.1.2/../../../../nios2-elf/lib/mno-hw-mul/libc.a(lib_a-memcpy.o)
 .debug_frame   0x00001114       0x20 /opt/altera/altera12.1/nios2eds/bin/gnu/H-i686-pc-linux-gnu/bin/../lib/gcc/nios2-elf/4.1.2/../../../../nios2-elf/lib/mno-hw-mul/libc.a(lib_a-strlen.o)
 .debug_frame   0x00001134       0x34 /opt/altera/altera12.1/nios2eds/bin/gnu/H-i686-pc-linux-gnu/bin/../lib/gcc/nios2-elf/4.1.2/../../../../nios2-elf/lib/mno-hw-mul/libc.a(lib_a-__atexit.o)
 .debug_frame   0x00001168       0x4c /opt/altera/altera12.1/nios2eds/bin/gnu/H-i686-pc-linux-gnu/bin/../lib/gcc/nios2-elf/4.1.2/../../../../nios2-elf/lib/mno-hw-mul/libc.a(lib_a-__call_atexit.o)
 .debug_frame   0x000011b4       0x48 ../snake_software_bsp//libhal_bsp.a(alt_exit.o)

.debug_str      0x00000000      0xd47
 *(.debug_str)
 .debug_str     0x00000000       0x12 obj/default/hello_world.o
 .debug_str     0x00000012      0x10a obj/default/main.o
 .debug_str     0x0000011c      0x169 /opt/altera/altera12.1/nios2eds/bin/gnu/H-i686-pc-linux-gnu/bin/../lib/gcc/nios2-elf/4.1.2/mno-hw-mul/libgcc.a(lib2-divmod.o)
                                0x1b6 (size before relaxing)
 .debug_str     0x00000285       0x37 /opt/altera/altera12.1/nios2eds/bin/gnu/H-i686-pc-linux-gnu/bin/../lib/gcc/nios2-elf/4.1.2/mno-hw-mul/libgcc.a(lib2-mul.o)
                                0x177 (size before relaxing)
 .debug_str     0x000002bc       0x12 ../snake_software_bsp//libhal_bsp.a(alt_load.o)
 .debug_str     0x000002ce       0x12 ../snake_software_bsp//libhal_bsp.a(alt_main.o)
 .debug_str     0x000002e0       0x12 ../snake_software_bsp//libhal_bsp.a(alt_usleep.o)
 .debug_str     0x000002f2       0x12 ../snake_software_bsp//libhal_bsp.a(alt_sys_init.o)
 .debug_str     0x00000304       0x12 ../snake_software_bsp//libhal_bsp.a(altera_avalon_jtag_uart_fd.o)
 .debug_str     0x00000316       0x1a ../snake_software_bsp//libhal_bsp.a(altera_avalon_jtag_uart_init.o)
 .debug_str     0x00000330       0x12 ../snake_software_bsp//libhal_bsp.a(altera_avalon_jtag_uart_ioctl.o)
 .debug_str     0x00000342       0x1a ../snake_software_bsp//libhal_bsp.a(altera_avalon_jtag_uart_read.o)
 .debug_str     0x0000035c       0x1a ../snake_software_bsp//libhal_bsp.a(altera_avalon_jtag_uart_write.o)
 .debug_str     0x00000376       0x23 ../snake_software_bsp//libhal_bsp.a(alt_alarm_start.o)
 .debug_str     0x00000399       0x12 ../snake_software_bsp//libhal_bsp.a(alt_busy_sleep.o)
 .debug_str     0x000003ab       0x12 ../snake_software_bsp//libhal_bsp.a(alt_close.o)
 .debug_str     0x000003bd       0x12 ../snake_software_bsp//libhal_bsp.a(alt_dcache_flush_all.o)
 .debug_str     0x000003cf       0x12 ../snake_software_bsp//libhal_bsp.a(alt_dev.o)
 .debug_str     0x000003e1       0x12 ../snake_software_bsp//libhal_bsp.a(alt_dev_llist_insert.o)
 .debug_str     0x000003f3       0x12 ../snake_software_bsp//libhal_bsp.a(alt_errno.o)
 .debug_str     0x00000405       0x12 ../snake_software_bsp//libhal_bsp.a(alt_icache_flush_all.o)
 .debug_str     0x00000417       0x18 ../snake_software_bsp//libhal_bsp.a(alt_iic.o)
 .debug_str     0x0000042f       0x1a ../snake_software_bsp//libhal_bsp.a(alt_iic_isr_register.o)
 .debug_str     0x00000449       0x12 ../snake_software_bsp//libhal_bsp.a(alt_io_redirect.o)
 .debug_str     0x0000045b       0x12 ../snake_software_bsp//libhal_bsp.a(alt_irq_handler.o)
 .debug_str     0x0000046d       0x12 ../snake_software_bsp//libhal_bsp.a(alt_open.o)
 .debug_str     0x0000047f       0x1a ../snake_software_bsp//libhal_bsp.a(alt_tick.o)
 .debug_str     0x00000499       0x12 ../snake_software_bsp//libhal_bsp.a(altera_nios2_irq.o)
 .debug_str     0x000004ab       0x12 ../snake_software_bsp//libhal_bsp.a(alt_find_dev.o)
 .debug_str     0x000004bd       0x12 ../snake_software_bsp//libhal_bsp.a(alt_find_file.o)
 .debug_str     0x000004cf       0x12 ../snake_software_bsp//libhal_bsp.a(alt_get_fd.o)
 .debug_str     0x000004e1      0x12d /opt/altera/altera12.1/nios2eds/bin/gnu/H-i686-pc-linux-gnu/bin/../lib/gcc/nios2-elf/4.1.2/../../../../nios2-elf/lib/mno-hw-mul/libc.a(lib_a-atexit.o)
                                0x1cf (size before relaxing)
 .debug_str     0x0000060e      0x387 /opt/altera/altera12.1/nios2eds/bin/gnu/H-i686-pc-linux-gnu/bin/../lib/gcc/nios2-elf/4.1.2/../../../../nios2-elf/lib/mno-hw-mul/libc.a(lib_a-exit.o)
                                0x51c (size before relaxing)
 .debug_str     0x00000995       0xe1 /opt/altera/altera12.1/nios2eds/bin/gnu/H-i686-pc-linux-gnu/bin/../lib/gcc/nios2-elf/4.1.2/../../../../nios2-elf/lib/mno-hw-mul/libc.a(lib_a-impure.o)
                                0x52a (size before relaxing)
 .debug_str     0x00000a76       0x40 /opt/altera/altera12.1/nios2eds/bin/gnu/H-i686-pc-linux-gnu/bin/../lib/gcc/nios2-elf/4.1.2/../../../../nios2-elf/lib/mno-hw-mul/libc.a(lib_a-int_errno.o)
                                0x173 (size before relaxing)
 .debug_str     0x00000ab6       0xe5 /opt/altera/altera12.1/nios2eds/bin/gnu/H-i686-pc-linux-gnu/bin/../lib/gcc/nios2-elf/4.1.2/../../../../nios2-elf/lib/mno-hw-mul/libc.a(lib_a-memcmp.o)
                                0x17a (size before relaxing)
 .debug_str     0x00000b9b       0x6c /opt/altera/altera12.1/nios2eds/bin/gnu/H-i686-pc-linux-gnu/bin/../lib/gcc/nios2-elf/4.1.2/../../../../nios2-elf/lib/mno-hw-mul/libc.a(lib_a-memcpy.o)
                                0x138 (size before relaxing)
 .debug_str     0x00000c07       0x52 /opt/altera/altera12.1/nios2eds/bin/gnu/H-i686-pc-linux-gnu/bin/../lib/gcc/nios2-elf/4.1.2/../../../../nios2-elf/lib/mno-hw-mul/libc.a(lib_a-strlen.o)
                                0x18d (size before relaxing)
 .debug_str     0x00000c59       0x54 /opt/altera/altera12.1/nios2eds/bin/gnu/H-i686-pc-linux-gnu/bin/../lib/gcc/nios2-elf/4.1.2/../../../../nios2-elf/lib/mno-hw-mul/libc.a(lib_a-__atexit.o)
                                0x534 (size before relaxing)
 .debug_str     0x00000cad       0x7e /opt/altera/altera12.1/nios2eds/bin/gnu/H-i686-pc-linux-gnu/bin/../lib/gcc/nios2-elf/4.1.2/../../../../nios2-elf/lib/mno-hw-mul/libc.a(lib_a-__call_atexit.o)
                                0x55e (size before relaxing)
 .debug_str     0x00000d2b       0x1c ../snake_software_bsp//libhal_bsp.a(alt_exit.o)

.debug_loc      0x00000000     0x1cb0
 *(.debug_loc)
 .debug_loc     0x00000000      0xcf4 obj/default/main.o
 .debug_loc     0x00000cf4      0x1d2 /opt/altera/altera12.1/nios2eds/bin/gnu/H-i686-pc-linux-gnu/bin/../lib/gcc/nios2-elf/4.1.2/mno-hw-mul/libgcc.a(lib2-divmod.o)
 .debug_loc     0x00000ec6       0x4f /opt/altera/altera12.1/nios2eds/bin/gnu/H-i686-pc-linux-gnu/bin/../lib/gcc/nios2-elf/4.1.2/mno-hw-mul/libgcc.a(lib2-mul.o)
 .debug_loc     0x00000f15       0x56 ../snake_software_bsp//libhal_bsp.a(alt_load.o)
 .debug_loc     0x00000f6b       0x2b ../snake_software_bsp//libhal_bsp.a(alt_main.o)
 .debug_loc     0x00000f96       0x2b ../snake_software_bsp//libhal_bsp.a(alt_usleep.o)
 .debug_loc     0x00000fc1       0x81 ../snake_software_bsp//libhal_bsp.a(alt_sys_init.o)
 .debug_loc     0x00001042       0xac ../snake_software_bsp//libhal_bsp.a(altera_avalon_jtag_uart_fd.o)
 .debug_loc     0x000010ee       0xac ../snake_software_bsp//libhal_bsp.a(altera_avalon_jtag_uart_init.o)
 .debug_loc     0x0000119a       0x2b ../snake_software_bsp//libhal_bsp.a(altera_avalon_jtag_uart_ioctl.o)
 .debug_loc     0x000011c5       0x2b ../snake_software_bsp//libhal_bsp.a(altera_avalon_jtag_uart_read.o)
 .debug_loc     0x000011f0       0x2b ../snake_software_bsp//libhal_bsp.a(altera_avalon_jtag_uart_write.o)
 .debug_loc     0x0000121b       0x2b ../snake_software_bsp//libhal_bsp.a(alt_alarm_start.o)
 .debug_loc     0x00001246       0x2b ../snake_software_bsp//libhal_bsp.a(alt_busy_sleep.o)
 .debug_loc     0x00001271       0x56 ../snake_software_bsp//libhal_bsp.a(alt_close.o)
 .debug_loc     0x000012c7       0x2b ../snake_software_bsp//libhal_bsp.a(alt_dcache_flush_all.o)
 .debug_loc     0x000012f2       0x2b ../snake_software_bsp//libhal_bsp.a(alt_dev.o)
 .debug_loc     0x0000131d       0x56 ../snake_software_bsp//libhal_bsp.a(alt_dev_llist_insert.o)
 .debug_loc     0x00001373       0x2b ../snake_software_bsp//libhal_bsp.a(alt_do_ctors.o)
 .debug_loc     0x0000139e       0x2b ../snake_software_bsp//libhal_bsp.a(alt_do_dtors.o)
 .debug_loc     0x000013c9       0x2b ../snake_software_bsp//libhal_bsp.a(alt_icache_flush_all.o)
 .debug_loc     0x000013f4       0xac ../snake_software_bsp//libhal_bsp.a(alt_iic.o)
 .debug_loc     0x000014a0       0x2b ../snake_software_bsp//libhal_bsp.a(alt_iic_isr_register.o)
 .debug_loc     0x000014cb       0x56 ../snake_software_bsp//libhal_bsp.a(alt_io_redirect.o)
 .debug_loc     0x00001521       0x2b ../snake_software_bsp//libhal_bsp.a(alt_irq_handler.o)
 .debug_loc     0x0000154c       0x81 ../snake_software_bsp//libhal_bsp.a(alt_open.o)
 .debug_loc     0x000015cd       0x2b ../snake_software_bsp//libhal_bsp.a(alt_release_fd.o)
 .debug_loc     0x000015f8       0x56 ../snake_software_bsp//libhal_bsp.a(alt_tick.o)
 .debug_loc     0x0000164e       0x2b ../snake_software_bsp//libhal_bsp.a(altera_nios2_irq.o)
 .debug_loc     0x00001679       0x2b ../snake_software_bsp//libhal_bsp.a(alt_find_dev.o)
 .debug_loc     0x000016a4       0x2b ../snake_software_bsp//libhal_bsp.a(alt_find_file.o)
 .debug_loc     0x000016cf       0x2b ../snake_software_bsp//libhal_bsp.a(alt_get_fd.o)
 .debug_loc     0x000016fa       0x1e /opt/altera/altera12.1/nios2eds/bin/gnu/H-i686-pc-linux-gnu/bin/../lib/gcc/nios2-elf/4.1.2/../../../../nios2-elf/lib/mno-hw-mul/libc.a(lib_a-atexit.o)
 .debug_loc     0x00001718       0x3d /opt/altera/altera12.1/nios2eds/bin/gnu/H-i686-pc-linux-gnu/bin/../lib/gcc/nios2-elf/4.1.2/../../../../nios2-elf/lib/mno-hw-mul/libc.a(lib_a-exit.o)
 .debug_loc     0x00001755      0x114 /opt/altera/altera12.1/nios2eds/bin/gnu/H-i686-pc-linux-gnu/bin/../lib/gcc/nios2-elf/4.1.2/../../../../nios2-elf/lib/mno-hw-mul/libc.a(lib_a-memcmp.o)
 .debug_loc     0x00001869       0xca /opt/altera/altera12.1/nios2eds/bin/gnu/H-i686-pc-linux-gnu/bin/../lib/gcc/nios2-elf/4.1.2/../../../../nios2-elf/lib/mno-hw-mul/libc.a(lib_a-memcpy.o)
 .debug_loc     0x00001933       0x3c /opt/altera/altera12.1/nios2eds/bin/gnu/H-i686-pc-linux-gnu/bin/../lib/gcc/nios2-elf/4.1.2/../../../../nios2-elf/lib/mno-hw-mul/libc.a(lib_a-strlen.o)
 .debug_loc     0x0000196f      0x120 /opt/altera/altera12.1/nios2eds/bin/gnu/H-i686-pc-linux-gnu/bin/../lib/gcc/nios2-elf/4.1.2/../../../../nios2-elf/lib/mno-hw-mul/libc.a(lib_a-__atexit.o)
 .debug_loc     0x00001a8f      0x1cb /opt/altera/altera12.1/nios2eds/bin/gnu/H-i686-pc-linux-gnu/bin/../lib/gcc/nios2-elf/4.1.2/../../../../nios2-elf/lib/mno-hw-mul/libc.a(lib_a-__call_atexit.o)
 .debug_loc     0x00001c5a       0x56 ../snake_software_bsp//libhal_bsp.a(alt_exit.o)

.debug_macinfo
 *(.debug_macinfo)

.debug_weaknames
 *(.debug_weaknames)

.debug_funcnames
 *(.debug_funcnames)

.debug_typenames
 *(.debug_typenames)

.debug_varnames
 *(.debug_varnames)

.debug_alt_sim_info
                0x00000000       0x40
 *(.debug_alt_sim_info)
 .debug_alt_sim_info
                0x00000000       0x10 ../snake_software_bsp//obj/HAL/src/crt0.o
 .debug_alt_sim_info
                0x00000010       0x30 ../snake_software_bsp//libhal_bsp.a(alt_busy_sleep.o)
                0x00100000                __alt_data_end = 0x100000
                0x00100000                PROVIDE (__alt_stack_pointer, __alt_data_end)
                0x0008fd98                PROVIDE (__alt_stack_limit, __alt_stack_base)
                0x0008fd98                PROVIDE (__alt_heap_start, end)
                0x00100000                PROVIDE (__alt_heap_limit, 0x100000)
OUTPUT(snake_software.elf elf32-littlenios2)

.debug_ranges   0x00000000       0x90
 .debug_ranges  0x00000000       0x20 ../snake_software_bsp//obj/HAL/src/crt0.o
 .debug_ranges  0x00000020       0x28 ../snake_software_bsp//libhal_bsp.a(alt_irq_entry.o)
 .debug_ranges  0x00000048       0x30 ../snake_software_bsp//libhal_bsp.a(alt_exception_entry.o)
 .debug_ranges  0x00000078       0x18 /opt/altera/altera12.1/nios2eds/bin/gnu/H-i686-pc-linux-gnu/bin/../lib/gcc/nios2-elf/4.1.2/../../../../nios2-elf/lib/mno-hw-mul/libc.a(lib_a-__call_atexit.o)
